 iterreachobj001

 Timestamp is 6a55e663 (reproducible build file hash)

 Preferred load address is 0000000180000000

 Start         Length     Name                   Class
 0001:00000000 00004ab0H .text$mn                CODE
 0001:00004ab0 00000036H .text$mn$00             CODE
 0001:00004ae6 00000092H .text$x                 CODE
 0002:00000000 000001c8H .idata$5                DATA
 0002:000001c8 00000038H .00cfg                  DATA
 0002:00000200 00000008H .CRT$XCA                DATA
 0002:00000208 00000008H .CRT$XCZ                DATA
 0002:00000210 00000008H .CRT$XIA                DATA
 0002:00000218 00000008H .CRT$XIC                DATA
 0002:00000220 00000008H .CRT$XIZ                DATA
 0002:00000228 00000008H .CRT$XLA                DATA
 0002:00000230 00000008H .CRT$XLZ                DATA
 0002:00000238 00000008H .CRT$XPA                DATA
 0002:00000240 00000008H .CRT$XPZ                DATA
 0002:00000248 00000008H .CRT$XTA                DATA
 0002:00000250 00000010H .CRT$XTZ                DATA
 0002:00000258 00000000H .gehcont$y              DATA
 0002:00000258 00000000H .gfids$y                DATA
 0002:00000260 000036a0H .rdata                  DATA
 0002:00003900 00000000H .rdata$CastGuardVftablesA DATA
 0002:00003900 00000000H .rdata$CastGuardVftablesC DATA
 0002:00003900 00000028H .rdata$T                DATA
 0002:00003928 000000bcH .rdata$voltmd           DATA
 0002:000039e4 0000031cH .rdata$zzzdbg           DATA
 0002:00003d00 00000008H .rtc$IAA                DATA
 0002:00003d08 00000008H .rtc$IZZ                DATA
 0002:00003d10 00000008H .rtc$TAA                DATA
 0002:00003d18 00000008H .rtc$TZZ                DATA
 0002:00003d20 00000004H .tls                    DATA
 0002:00003d24 00000004H .tls$                   DATA
 0002:00003d28 00000008H .tls$ZZZ                DATA
 0002:00003d30 00000400H .xdata                  DATA
 0002:00004130 00000368H .edata                  DATA
 0002:00004498 0000008cH .idata$2                DATA
 0002:00004524 00000014H .idata$3                DATA
 0002:00004538 000001c8H .idata$4                DATA
 0002:00004700 00000486H .idata$6                DATA
 0003:00000000 00000080H .data                   DATA
 0003:00000080 0001b248H .bss                    DATA
 0004:00000000 0000042cH .pdata                  DATA

  Address         Publics by Value              Rva+Base               Lib:Object

 0000:00000000       __AbsoluteZero             0000000000000000     <absolute>
 0000:00000000       ___safe_se_handler_count   0000000000000000     <absolute>
 0000:00000000       ___safe_se_handler_table   0000000000000000     <absolute>
 0000:00000000       __arm64x_extra_rfe_table   0000000000000000     <absolute>
 0000:00000000       __arm64x_extra_rfe_table_size 0000000000000000     <absolute>
 0000:00000000       __arm64x_native_entrypoint 0000000000000000     <absolute>
 0000:00000000       __arm64x_redirection_metadata 0000000000000000     <absolute>
 0000:00000000       __arm64x_redirection_metadata_count 0000000000000000     <absolute>
 0000:00000000       __dynamic_value_reloc_table 0000000000000000     <absolute>
 0000:00000000       __enclave_config           0000000000000000     <absolute>
 0000:00000000       __guard_check_icall_a64n_fptr 0000000000000000     <absolute>
 0000:00000000       __guard_eh_cont_count      0000000000000000     <absolute>
 0000:00000000       __guard_eh_cont_table      0000000000000000     <absolute>
 0000:00000000       __guard_fids_count         0000000000000000     <absolute>
 0000:00000000       __guard_fids_table         0000000000000000     <absolute>
 0000:00000000       __guard_iat_count          0000000000000000     <absolute>
 0000:00000000       __guard_iat_table          0000000000000000     <absolute>
 0000:00000000       __guard_longjmp_count      0000000000000000     <absolute>
 0000:00000000       __guard_longjmp_table      0000000000000000     <absolute>
 0000:00000000       __hybrid_auxiliary_iat     0000000000000000     <absolute>
 0000:00000000       __hybrid_auxiliary_iat_copy 0000000000000000     <absolute>
 0000:00000000       __hybrid_code_map          0000000000000000     <absolute>
 0000:00000000       __hybrid_code_map_count    0000000000000000     <absolute>
 0000:00000000       __x64_code_ranges_to_entry_points 0000000000000000     <absolute>
 0000:00000000       __x64_code_ranges_to_entry_points_count 0000000000000000     <absolute>
 0000:00000100       __guard_flags              0000000000000100     <absolute>
 0000:00000000       __ImageBase                0000000180000000     <linker-defined>
 0001:00000000       ?NewObject@JNIEnv_@@QEAAPEAV_jobject@@PEAV_jclass@@PEAU_jmethodID@@ZZ 0000000180001000 f i libiterreachobj001.obj
 0001:00000028       ?TranslateError@@YAPEBDW4jvmtiError@@@Z 0000000180001028 f   libiterreachobj001.obj
 0001:000002e0       ?nsk_jni_check_exception@@YAHPEAUJNIEnv_@@QEBDH@Z 00000001800012e0 f   libiterreachobj001.obj
 0001:00000424       ?nsk_jni_lverify@@YAHHPEAUJNIEnv_@@HQEBDH1ZZ 0000000180001424 f   libiterreachobj001.obj
 0001:000004c4       Agent_Initialize           00000001800014c4 f   libiterreachobj001.obj
 0001:000007f4       Agent_OnAttach             00000001800017f4 f   libiterreachobj001.obj
 0001:000007f4       Agent_OnLoad               00000001800017f4 f   libiterreachobj001.obj
 0001:000007fc       Java_nsk_jvmti_unit_FollowReferences_FollowRefObjects_addRefToVerify 00000001800017fc f   libiterreachobj001.obj
 0001:000009d4       Java_nsk_jvmti_unit_FollowReferences_FollowRefObjects_getTag 00000001800019d4 f   libiterreachobj001.obj
 0001:00000a94       Java_nsk_jvmti_unit_FollowReferences_FollowRefObjects_resetRefsToVerify 0000000180001a94 f   libiterreachobj001.obj
 0001:00000a9c       Java_nsk_jvmti_unit_FollowReferences_FollowRefObjects_resetTags 0000000180001a9c f   libiterreachobj001.obj
 0001:00000ae0       Java_nsk_jvmti_unit_FollowReferences_FollowRefObjects_setTag 0000000180001ae0 f   libiterreachobj001.obj
 0001:00000d38       Java_nsk_share_jvmti_ArgumentHandler_getAgentOptionsString 0000000180001d38 f   libiterreachobj001.obj
 0001:00000de8       Java_nsk_share_jvmti_DebugeeClass_checkStatus 0000000180001de8 f   libiterreachobj001.obj
 0001:00000e70       Java_nsk_share_jvmti_DebugeeClass_resetAgentData 0000000180001e70 f   libiterreachobj001.obj
 0001:00000ed0       Java_nsk_share_jvmti_RedefineAgent_agentStatus 0000000180001ed0 f   libiterreachobj001.obj
 0001:00000edc       Java_nsk_share_jvmti_RedefineAgent_isRedefined 0000000180001edc f   libiterreachobj001.obj
 0001:00000ee8       Java_nsk_share_jvmti_RedefineAgent_redefineAttempted 0000000180001ee8 f   libiterreachobj001.obj
 0001:00000ef4       MA_checkStatus             0000000180001ef4 f   libiterreachobj001.obj
 0001:00000f98       __local_stdio_printf_options 0000000180001f98 f i libiterreachobj001.obj
 0001:00001828       exitOnError                0000000180002828 f   libiterreachobj001.obj
 0001:000018dc       fprintf                    00000001800028dc f i libiterreachobj001.obj
 0001:0000239c       heapRootCallback           000000018000339c f   libiterreachobj001.obj
 0001:0000255c       nsk_complain               000000018000355c f   libiterreachobj001.obj
 0001:00002588       nsk_jvmti_createJVMTIEnv   0000000180003588 f   libiterreachobj001.obj
 0001:000026b8       nsk_jvmti_findOptionIntValue 00000001800036b8 f   libiterreachobj001.obj
 0001:00002754       nsk_jvmti_findOptionValue  0000000180003754 f   libiterreachobj001.obj
 0001:000027cc       nsk_jvmti_lverify          00000001800037cc f   libiterreachobj001.obj
 0001:000028bc       nsk_jvmti_parseOptions     00000001800038bc f   libiterreachobj001.obj
 0001:00002b0c       nsk_jvmti_resetAgentData   0000000180003b0c f   libiterreachobj001.obj
 0001:00002b8c       nsk_jvmti_resumeSync       0000000180003b8c f   libiterreachobj001.obj
 0001:00002c34       nsk_jvmti_setFailStatus    0000000180003c34 f   libiterreachobj001.obj
 0001:00002c70       nsk_jvmti_waitForSync      0000000180003c70 f   libiterreachobj001.obj
 0001:00002d74       nsk_lcomplain              0000000180003d74 f   libiterreachobj001.obj
 0001:00002d94       nsk_ldisplay               0000000180003d94 f   libiterreachobj001.obj
 0001:00002db4       nsk_ltrace                 0000000180003db4 f   libiterreachobj001.obj
 0001:00002dd4       nsk_lvcomplain             0000000180003dd4 f   libiterreachobj001.obj
 0001:00002f8c       nsk_lvdisplay              0000000180003f8c f   libiterreachobj001.obj
 0001:00002fd8       nsk_lverify                0000000180003fd8 f   libiterreachobj001.obj
 0001:00003034       nsk_lvtrace                0000000180004034 f   libiterreachobj001.obj
 0001:00003094       nsk_printf                 0000000180004094 f   libiterreachobj001.obj
 0001:000030bc       nsk_vprintf                00000001800040bc f   libiterreachobj001.obj
 0001:00003170       objectReferenceCallback    0000000180004170 f   libiterreachobj001.obj
 0001:0000334c       printf                     000000018000434c f i libiterreachobj001.obj
 0001:00003464       stackReferenceCallback     0000000180004464 f   libiterreachobj001.obj
 0001:00003b90       __raise_securityfailure    0000000180004b90 f   MSVCRT:gs_report.obj
 0001:00003bc4       __report_gsfailure         0000000180004bc4 f   MSVCRT:gs_report.obj
 0001:00003e04       __GSHandlerCheck           0000000180004e04 f   MSVCRT:gshandler.obj
 0001:00003e24       __GSHandlerCheckCommon     0000000180004e24 f   MSVCRT:gshandler.obj
 0001:00003e90       __security_check_cookie    0000000180004e90 f   MSVCRT:amdsecgs.obj
 0001:000041d0       _DllMainCRTStartup         00000001800051d0 f   MSVCRT:dll_dllmain.obj
 0001:00004210       __scrt_acquire_startup_lock 0000000180005210 f   MSVCRT:utility.obj
 0001:0000424c       __scrt_dllmain_after_initialize_c 000000018000524c f   MSVCRT:utility.obj
 0001:00004280       __scrt_dllmain_before_initialize_c 0000000180005280 f   MSVCRT:utility.obj
 0001:00004298       __scrt_dllmain_crt_thread_attach 0000000180005298 f   MSVCRT:utility.obj
 0001:000042c0       __scrt_dllmain_crt_thread_detach 00000001800052c0 f   MSVCRT:utility.obj
 0001:000042d8       __scrt_dllmain_exception_filter 00000001800052d8 f   MSVCRT:utility.obj
 0001:00004338       __scrt_dllmain_uninitialize_c 0000000180005338 f   MSVCRT:utility.obj
 0001:00004368       __scrt_dllmain_uninitialize_critical 0000000180005368 f   MSVCRT:utility.obj
 0001:0000437c       __scrt_initialize_crt      000000018000537c f   MSVCRT:utility.obj
 0001:000043c8       __scrt_initialize_onexit_tables 00000001800053c8 f   MSVCRT:utility.obj
 0001:00004454       __scrt_is_nonwritable_in_current_image 0000000180005454 f   MSVCRT:utility.obj
 0001:000044ec       __scrt_release_startup_lock 00000001800054ec f   MSVCRT:utility.obj
 0001:00004510       __scrt_uninitialize_crt    0000000180005510 f   MSVCRT:utility.obj
 0001:0000453c       _onexit                    000000018000553c f   MSVCRT:utility.obj
 0001:00004578       atexit                     0000000180005578 f   MSVCRT:utility.obj
 0001:00004590       __crt_debugger_hook        0000000180005590 f   MSVCRT:utility_desktop.obj
 0001:00004598       __scrt_fastfail            0000000180005598 f   MSVCRT:utility_desktop.obj
 0001:000046e4       _guard_check_icall_nop     00000001800056e4 f i MSVCRT:guard_support.obj
 0001:000046e8       __security_init_cookie     00000001800056e8 f   MSVCRT:gs_support.obj
 0001:00004794       DllMain                    0000000180005794 f   MSVCRT:dll_dllmain_stub.obj
 0001:000047b8       ?__scrt_initialize_type_info@@YAXXZ 00000001800057b8 f   MSVCRT:tncleanup.obj
 0001:000047c8       ?__scrt_uninitialize_type_info@@YAXXZ 00000001800057c8 f   MSVCRT:tncleanup.obj
 0001:000047d4       __local_stdio_scanf_options 00000001800057d4 f i MSVCRT:default_local_stdio_options.obj
 0001:000047dc       __scrt_initialize_default_local_stdio_options 00000001800057dc f   MSVCRT:default_local_stdio_options.obj
 0001:000047f8       __scrt_get_dyn_tls_init_callback 00000001800057f8 f   MSVCRT:dyn_tls_init.obj
 0001:00004800       _RTC_Initialize            0000000180005800 f   MSVCRT:initsect.obj
 0001:0000483c       _RTC_Terminate             000000018000583c f   MSVCRT:initsect.obj
 0001:00004878       __isa_available_init       0000000180005878 f   MSVCRT:cpu_disp.obj
 0001:00004a24       _get_startup_argv_mode     0000000180005a24 f   MSVCRT:argv_mode.obj
 0001:00004a2c       __scrt_is_ucrt_dll_in_use  0000000180005a2c f   MSVCRT:ucrt_detection.obj
 0001:00004a40       memcpy                     0000000180005a40 f   vcruntime:VCRUNTIME140.dll
 0001:00004a46       memset                     0000000180005a46 f   vcruntime:VCRUNTIME140.dll
 0001:00004a4c       strchr                     0000000180005a4c f   vcruntime:VCRUNTIME140.dll
 0001:00004a52       __C_specific_handler       0000000180005a52 f   vcruntime:VCRUNTIME140.dll
 0001:00004a58       __std_type_info_destroy_list 0000000180005a58 f   vcruntime:VCRUNTIME140.dll
 0001:00004a5e       strcmp                     0000000180005a5e f   ucrt:api-ms-win-crt-string-l1-1-0.dll
 0001:00004a64       strlen                     0000000180005a64 f   ucrt:api-ms-win-crt-string-l1-1-0.dll
 0001:00004a6a       _initterm                  0000000180005a6a f   ucrt:api-ms-win-crt-runtime-l1-1-0.dll
 0001:00004a70       _initterm_e                0000000180005a70 f   ucrt:api-ms-win-crt-runtime-l1-1-0.dll
 0001:00004a76       _seh_filter_dll            0000000180005a76 f   ucrt:api-ms-win-crt-runtime-l1-1-0.dll
 0001:00004a7c       _configure_narrow_argv     0000000180005a7c f   ucrt:api-ms-win-crt-runtime-l1-1-0.dll
 0001:00004a82       _initialize_narrow_environment 0000000180005a82 f   ucrt:api-ms-win-crt-runtime-l1-1-0.dll
 0001:00004a88       _initialize_onexit_table   0000000180005a88 f   ucrt:api-ms-win-crt-runtime-l1-1-0.dll
 0001:00004a8e       _register_onexit_function  0000000180005a8e f   ucrt:api-ms-win-crt-runtime-l1-1-0.dll
 0001:00004a94       _execute_onexit_table      0000000180005a94 f   ucrt:api-ms-win-crt-runtime-l1-1-0.dll
 0001:00004a9a       _crt_atexit                0000000180005a9a f   ucrt:api-ms-win-crt-runtime-l1-1-0.dll
 0001:00004aa0       _cexit                     0000000180005aa0 f   ucrt:api-ms-win-crt-runtime-l1-1-0.dll
 0001:00004aa8       __acrt_initialize          0000000180005aa8 f   MSVCRT:ucrt_stubs.obj
 0001:00004aa8       __acrt_thread_attach       0000000180005aa8 f   MSVCRT:ucrt_stubs.obj
 0001:00004aa8       __acrt_thread_detach       0000000180005aa8 f   MSVCRT:ucrt_stubs.obj
 0001:00004aa8       __acrt_uninitialize        0000000180005aa8 f   MSVCRT:ucrt_stubs.obj
 0001:00004aa8       __acrt_uninitialize_critical 0000000180005aa8 f   MSVCRT:ucrt_stubs.obj
 0001:00004aa8       __scrt_stub_for_acrt_initialize 0000000180005aa8 f   MSVCRT:ucrt_stubs.obj
 0001:00004aa8       __scrt_stub_for_acrt_thread_attach 0000000180005aa8 f   MSVCRT:ucrt_stubs.obj
 0001:00004aa8       __scrt_stub_for_acrt_thread_detach 0000000180005aa8 f   MSVCRT:ucrt_stubs.obj
 0001:00004aa8       __scrt_stub_for_acrt_uninitialize 0000000180005aa8 f   MSVCRT:ucrt_stubs.obj
 0001:00004aa8       __scrt_stub_for_acrt_uninitialize_critical 0000000180005aa8 f   MSVCRT:ucrt_stubs.obj
 0001:00004aa8       __vcrt_initialize          0000000180005aa8 f   MSVCRT:ucrt_stubs.obj
 0001:00004aa8       __vcrt_thread_attach       0000000180005aa8 f   MSVCRT:ucrt_stubs.obj
 0001:00004aa8       __vcrt_thread_detach       0000000180005aa8 f   MSVCRT:ucrt_stubs.obj
 0001:00004aa8       __vcrt_uninitialize        0000000180005aa8 f   MSVCRT:ucrt_stubs.obj
 0001:00004aa8       __vcrt_uninitialize_critical 0000000180005aa8 f   MSVCRT:ucrt_stubs.obj
 0001:00004aac       __scrt_stub_for_is_c_termination_complete 0000000180005aac f   MSVCRT:ucrt_stubs.obj
 0001:00004aac       _is_c_termination_complete 0000000180005aac f   MSVCRT:ucrt_stubs.obj
 0001:00004ac0       _guard_dispatch_icall_nop  0000000180005ac0 f   MSVCRT:guard_dispatch.obj
 0001:00004ae0       _guard_xfg_dispatch_icall_nop 0000000180005ae0 f   MSVCRT:guard_xfg_dispatch.obj
 0002:00000000       __imp_RtlCaptureContext    0000000180006000     kernel32:KERNEL32.dll
 0002:00000008       __imp_RtlLookupFunctionEntry 0000000180006008     kernel32:KERNEL32.dll
 0002:00000010       __imp_RtlVirtualUnwind     0000000180006010     kernel32:KERNEL32.dll
 0002:00000018       __imp_UnhandledExceptionFilter 0000000180006018     kernel32:KERNEL32.dll
 0002:00000020       __imp_SetUnhandledExceptionFilter 0000000180006020     kernel32:KERNEL32.dll
 0002:00000028       __imp_GetCurrentProcess    0000000180006028     kernel32:KERNEL32.dll
 0002:00000030       __imp_TerminateProcess     0000000180006030     kernel32:KERNEL32.dll
 0002:00000038       __imp_IsProcessorFeaturePresent 0000000180006038     kernel32:KERNEL32.dll
 0002:00000040       __imp_CloseHandle          0000000180006040     kernel32:KERNEL32.dll
 0002:00000048       __imp_InitializeCriticalSectionAndSpinCount 0000000180006048     kernel32:KERNEL32.dll
 0002:00000050       __imp_DeleteCriticalSection 0000000180006050     kernel32:KERNEL32.dll
 0002:00000058       __imp_CreateEventW         0000000180006058     kernel32:KERNEL32.dll
 0002:00000060       __imp_GetModuleHandleW     0000000180006060     kernel32:KERNEL32.dll
 0002:00000068       __imp_GetProcAddress       0000000180006068     kernel32:KERNEL32.dll
 0002:00000070       __imp_IsDebuggerPresent    0000000180006070     kernel32:KERNEL32.dll
 0002:00000078       __imp_QueryPerformanceCounter 0000000180006078     kernel32:KERNEL32.dll
 0002:00000080       __imp_GetCurrentProcessId  0000000180006080     kernel32:KERNEL32.dll
 0002:00000088       __imp_GetCurrentThreadId   0000000180006088     kernel32:KERNEL32.dll
 0002:00000090       __imp_GetSystemTimeAsFileTime 0000000180006090     kernel32:KERNEL32.dll
 0002:00000098       __imp_DisableThreadLibraryCalls 0000000180006098     kernel32:KERNEL32.dll
 0002:000000a0       __imp_InitializeSListHead  00000001800060a0     kernel32:KERNEL32.dll
 0002:000000a8       \177KERNEL32_NULL_THUNK_DATA 00000001800060a8     kernel32:KERNEL32.dll
 0002:000000b0       __imp_memcpy               00000001800060b0     vcruntime:VCRUNTIME140.dll
 0002:000000b8       __imp_memset               00000001800060b8     vcruntime:VCRUNTIME140.dll
 0002:000000c0       __imp_strchr               00000001800060c0     vcruntime:VCRUNTIME140.dll
 0002:000000c8       __imp___C_specific_handler 00000001800060c8     vcruntime:VCRUNTIME140.dll
 0002:000000d0       __imp___std_type_info_destroy_list 00000001800060d0     vcruntime:VCRUNTIME140.dll
 0002:000000d8       \177VCRUNTIME140_NULL_THUNK_DATA 00000001800060d8     vcruntime:VCRUNTIME140.dll
 0002:000000e0       __imp_strtol               00000001800060e0     ucrt:api-ms-win-crt-convert-l1-1-0.dll
 0002:000000e8       \177api-ms-win-crt-convert-l1-1-0_NULL_THUNK_DATA 00000001800060e8     ucrt:api-ms-win-crt-convert-l1-1-0.dll
 0002:000000f0       __imp_malloc               00000001800060f0     ucrt:api-ms-win-crt-heap-l1-1-0.dll
 0002:000000f8       __imp_free                 00000001800060f8     ucrt:api-ms-win-crt-heap-l1-1-0.dll
 0002:00000100       \177api-ms-win-crt-heap-l1-1-0_NULL_THUNK_DATA 0000000180006100     ucrt:api-ms-win-crt-heap-l1-1-0.dll
 0002:00000108       __imp__errno               0000000180006108     ucrt:api-ms-win-crt-runtime-l1-1-0.dll
 0002:00000110       __imp_exit                 0000000180006110     ucrt:api-ms-win-crt-runtime-l1-1-0.dll
 0002:00000118       __imp__cexit               0000000180006118     ucrt:api-ms-win-crt-runtime-l1-1-0.dll
 0002:00000120       __imp__crt_atexit          0000000180006120     ucrt:api-ms-win-crt-runtime-l1-1-0.dll
 0002:00000128       __imp__execute_onexit_table 0000000180006128     ucrt:api-ms-win-crt-runtime-l1-1-0.dll
 0002:00000130       __imp__register_onexit_function 0000000180006130     ucrt:api-ms-win-crt-runtime-l1-1-0.dll
 0002:00000138       __imp__initialize_onexit_table 0000000180006138     ucrt:api-ms-win-crt-runtime-l1-1-0.dll
 0002:00000140       __imp__initialize_narrow_environment 0000000180006140     ucrt:api-ms-win-crt-runtime-l1-1-0.dll
 0002:00000148       __imp__configure_narrow_argv 0000000180006148     ucrt:api-ms-win-crt-runtime-l1-1-0.dll
 0002:00000150       __imp__seh_filter_dll      0000000180006150     ucrt:api-ms-win-crt-runtime-l1-1-0.dll
 0002:00000158       __imp__initterm_e          0000000180006158     ucrt:api-ms-win-crt-runtime-l1-1-0.dll
 0002:00000160       __imp__initterm            0000000180006160     ucrt:api-ms-win-crt-runtime-l1-1-0.dll
 0002:00000168       \177api-ms-win-crt-runtime-l1-1-0_NULL_THUNK_DATA 0000000180006168     ucrt:api-ms-win-crt-runtime-l1-1-0.dll
 0002:00000170       __imp___acrt_iob_func      0000000180006170     ucrt:api-ms-win-crt-stdio-l1-1-0.dll
 0002:00000178       __imp_fflush               0000000180006178     ucrt:api-ms-win-crt-stdio-l1-1-0.dll
 0002:00000180       __imp___stdio_common_vsprintf 0000000180006180     ucrt:api-ms-win-crt-stdio-l1-1-0.dll
 0002:00000188       __imp___stdio_common_vfprintf 0000000180006188     ucrt:api-ms-win-crt-stdio-l1-1-0.dll
 0002:00000190       \177api-ms-win-crt-stdio-l1-1-0_NULL_THUNK_DATA 0000000180006190     ucrt:api-ms-win-crt-stdio-l1-1-0.dll
 0002:00000198       __imp_strcmp               0000000180006198     ucrt:api-ms-win-crt-string-l1-1-0.dll
 0002:000001a0       __imp__strdup              00000001800061a0     ucrt:api-ms-win-crt-string-l1-1-0.dll
 0002:000001a0       __imp_strdup               00000001800061a0     ucrt:api-ms-win-crt-string-l1-1-0.dll
 0002:000001a8       __imp_strlen               00000001800061a8     ucrt:api-ms-win-crt-string-l1-1-0.dll
 0002:000001b0       __imp_strpbrk              00000001800061b0     ucrt:api-ms-win-crt-string-l1-1-0.dll
 0002:000001b8       __imp_strncpy              00000001800061b8     ucrt:api-ms-win-crt-string-l1-1-0.dll
 0002:000001c0       \177api-ms-win-crt-string-l1-1-0_NULL_THUNK_DATA 00000001800061c0     ucrt:api-ms-win-crt-string-l1-1-0.dll
 0002:000001c8       __guard_check_icall_fptr   00000001800061c8     MSVCRT:guard_support.obj
 0002:000001d0       __guard_xfg_check_icall_fptr 00000001800061d0     MSVCRT:guard_support.obj
 0002:000001d8       __guard_dispatch_icall_fptr 00000001800061d8     MSVCRT:guard_support.obj
 0002:000001e0       __guard_xfg_dispatch_icall_fptr 00000001800061e0     MSVCRT:guard_support.obj
 0002:000001e8       __guard_xfg_table_dispatch_icall_fptr 00000001800061e8     MSVCRT:guard_support.obj
 0002:000001f0       __castguard_check_failure_os_handled_fptr 00000001800061f0     MSVCRT:guard_support.obj
 0002:000001f8       __guard_memcpy_fptr        00000001800061f8     vcruntime:softmemtag.obj
 0002:00000200       __xc_a                     0000000180006200     MSVCRT:initializers.obj
 0002:00000208       __xc_z                     0000000180006208     MSVCRT:initializers.obj
 0002:00000210       __xi_a                     0000000180006210     MSVCRT:initializers.obj
 0002:00000220       __xi_z                     0000000180006220     MSVCRT:initializers.obj
 0002:00000228       __xl_a                     0000000180006228     MSVCRT:tlssup.obj
 0002:00000230       __xl_z                     0000000180006230     MSVCRT:tlssup.obj
 0002:00000238       __xp_a                     0000000180006238     MSVCRT:initializers.obj
 0002:00000240       __xp_z                     0000000180006240     MSVCRT:initializers.obj
 0002:00000248       __xt_a                     0000000180006248     MSVCRT:initializers.obj
 0002:00000250       __xt_z                     0000000180006250     MSVCRT:initializers.obj
 0002:00000260       g_refKindStr               0000000180006260     libiterreachobj001.obj
 0002:00000410       ??_C@_09BPLDFGCI@unknown_0@ 0000000180006410     libiterreachobj001.obj
 0002:00000420       ??_C@_0BL@FPNMECJD@JVMTI_HEAP_REFERENCE_CLASS@ 0000000180006420     libiterreachobj001.obj
 0002:00000440       ??_C@_0BL@FKGKKLNM@JVMTI_HEAP_REFERENCE_FIELD@ 0000000180006440     libiterreachobj001.obj
 0002:00000460       ??_C@_0CD@CAEHCFJF@JVMTI_HEAP_REFERENCE_ARRAY_ELEM@ 0000000180006460     libiterreachobj001.obj
 0002:00000488       ??_C@_0CC@DNEBMCNK@JVMTI_HEAP_REFERENCE_CLASS_LOAD@ 0000000180006488     libiterreachobj001.obj
 0002:000004b0       ??_C@_0BN@CJMIPEBB@JVMTI_HEAP_REFERENCE_SIGNERS@ 00000001800064b0     libiterreachobj001.obj
 0002:000004d0       ??_C@_0CH@HBOIDPEB@JVMTI_HEAP_REFERENCE_PROTECTION@ 00000001800064d0     libiterreachobj001.obj
 0002:000004f8       ??_C@_0BP@MDKGDGKL@JVMTI_HEAP_REFERENCE_INTERFACE@ 00000001800064f8     libiterreachobj001.obj
 0002:00000518       ??_C@_0CC@JJMIHNJH@JVMTI_HEAP_REFERENCE_STATIC_FIE@ 0000000180006518     libiterreachobj001.obj
 0002:00000540       ??_C@_0CD@IDHEEGID@JVMTI_HEAP_REFERENCE_CONSTANT_P@ 0000000180006540     libiterreachobj001.obj
 0002:00000568       ??_C@_0CA@EFFCHNG@JVMTI_HEAP_REFERENCE_SUPERCLASS@ 0000000180006568     libiterreachobj001.obj
 0002:00000588       ??_C@_0L@PCDFHGCJ@unknown_11@ 0000000180006588     libiterreachobj001.obj
 0002:00000598       ??_C@_0L@NJBICFOK@unknown_12@ 0000000180006598     libiterreachobj001.obj
 0002:000005a8       ??_C@_0L@MAADBEKL@unknown_13@ 00000001800065a8     libiterreachobj001.obj
 0002:000005b8       ??_C@_0L@IPECICGM@unknown_14@ 00000001800065b8     libiterreachobj001.obj
 0002:000005c8       ??_C@_0L@JGFJLDCN@unknown_15@ 00000001800065c8     libiterreachobj001.obj
 0002:000005d8       ??_C@_0L@LNHEOAOO@unknown_16@ 00000001800065d8     libiterreachobj001.obj
 0002:000005e8       ??_C@_0L@KEGPNBKP@unknown_17@ 00000001800065e8     libiterreachobj001.obj
 0002:000005f8       ??_C@_0L@CDPHMNGA@unknown_18@ 00000001800065f8     libiterreachobj001.obj
 0002:00000608       ??_C@_0L@DKOMPMCB@unknown_19@ 0000000180006608     libiterreachobj001.obj
 0002:00000618       ??_C@_0L@OJGIPJDB@unknown_20@ 0000000180006618     libiterreachobj001.obj
 0002:00000628       ??_C@_0CA@KAOFNDEM@JVMTI_HEAP_REFERENCE_JNI_GLOBAL@ 0000000180006628     libiterreachobj001.obj
 0002:00000648       ??_C@_0CC@HPFAJBK@JVMTI_HEAP_REFERENCE_SYSTEM_CLA@ 0000000180006648     libiterreachobj001.obj
 0002:00000670       ??_C@_0BN@FDEGFOHC@JVMTI_HEAP_REFERENCE_MONITOR@ 0000000180006670     libiterreachobj001.obj
 0002:00000690       ??_C@_0CB@HKIBCMAJ@JVMTI_HEAP_REFERENCE_STACK_LOCA@ 0000000180006690     libiterreachobj001.obj
 0002:000006b8       ??_C@_0BP@EAACMMOE@JVMTI_HEAP_REFERENCE_JNI_LOCAL@ 00000001800066b8     libiterreachobj001.obj
 0002:000006d8       ??_C@_0BM@IJDEOGOE@JVMTI_HEAP_REFERENCE_THREAD@ 00000001800066d8     libiterreachobj001.obj
 0002:000006f8       ??_C@_0BL@EDGPPKC@JVMTI_HEAP_REFERENCE_OTHER@ 00000001800066f8     libiterreachobj001.obj
 0002:00000714       ??_C@_04BCJPDBDA@Code@     0000000180006714     libiterreachobj001.obj
 0002:00000720       ??_C@_0BA@OCLMCFKC@LineNumberTable@ 0000000180006720     libiterreachobj001.obj
 0002:00000730       ??_C@_0BD@CPAEPILC@LocalVariableTable@ 0000000180006730     libiterreachobj001.obj
 0002:00000748       ??_C@_0BH@NMBDNHBD@LocalVariableTypeTable@ 0000000180006748     libiterreachobj001.obj
 0002:00000760       ??_C@_0O@HIHEEDNJ@StackMapTable@ 0000000180006760     libiterreachobj001.obj
 0002:00000770       ??_C@_0L@HCDIAMJG@?9?5?$CFs?0?5?$CFd?3?5@ 0000000180006770     libiterreachobj001.obj
 0002:00000780       ??_C@_0JI@HLPECLFI@?$CD?5?4?4?4?6?$CD?5ERROR?3?5too?5many?5complai@ 0000000180006780     libiterreachobj001.obj
 0002:00000820       ??_C@_0ED@JNEKCCOB@The?5following?5fake?5exception?5st@ 0000000180006820     libiterreachobj001.obj
 0002:00000868       ??_C@_0CN@FCNMDFBH@nsk?4share?4Fake_Exception_for_RU@ 0000000180006868     libiterreachobj001.obj
 0002:00000898       ??_C@_08PGFFNAEI@?$CI?$CFs?3?$CFd?$CJ?5@ 0000000180006898     libiterreachobj001.obj
 0002:000008a8       ??_C@_0DP@IENMAEGI@s?2test?2hotspot?2jtreg?2vmTestbase@ 00000001800068a8     libiterreachobj001.obj
 0002:000008e8       ??_C@_0BL@NDJLFFJB@?7at?5nsk_lvcomplain?$CI?$CFs?3?$CFd?$CJ?6@ 00000001800068e8     libiterreachobj001.obj
 0002:00000908       ??_C@_0BC@JOOKAFKF@?$CD?5ERROR?3?5?$CFs?0?5?$CFd?3?5@ 0000000180006908     libiterreachobj001.obj
 0002:00000920       ??_C@_09KJEAHMEH@?$CD?5ERROR?3?5@ 0000000180006920     libiterreachobj001.obj
 0002:0000092c       ??_C@_02GPIOPFAK@?$DO?$DO@ 000000018000692c     libiterreachobj001.obj
 0002:00000930       ??_C@_02FODMEDOG@?$DM?$DM@ 0000000180006930     libiterreachobj001.obj
 0002:00000934       ??_C@_02DJGKEECL@?4?4@     0000000180006934     libiterreachobj001.obj
 0002:00000938       ??_C@_0O@CJPGJOAF@?9?5?$CFs?0?5?$CFd?3?5?$CFs?5@ 0000000180006938     libiterreachobj001.obj
 0002:00000948       ??_C@_0CB@IAKPDOIC@?$CD?5?5?5verified?5assertion?5is?5FALSE@ 0000000180006948     libiterreachobj001.obj
 0002:00000970       ??_C@_0CO@LGONDEPD@stdout?3?5fflush?5failed?5?9?5err?$DN?$CFd?5@ 0000000180006970     libiterreachobj001.obj
 0002:000009a0       ??_C@_0CO@KBGKJPBD@stderr?3?5fflush?5failed?5?9?5err?$DN?$CFd?5@ 00000001800069a0     libiterreachobj001.obj
 0002:000009d0       ??_C@_0BB@JCNMKLLK@JVMTI_ERROR_NONE@ 00000001800069d0     libiterreachobj001.obj
 0002:000009e8       ??_C@_0BL@LDIMKLPH@JVMTI_ERROR_INVALID_THREAD@ 00000001800069e8     libiterreachobj001.obj
 0002:00000a08       ??_C@_0CB@PJFPAIKJ@JVMTI_ERROR_INVALID_THREAD_GROU@ 0000000180006a08     libiterreachobj001.obj
 0002:00000a30       ??_C@_0BN@LLMKHMNF@JVMTI_ERROR_INVALID_PRIORITY@ 0000000180006a30     libiterreachobj001.obj
 0002:00000a50       ??_C@_0CB@MBOFKAGB@JVMTI_ERROR_THREAD_NOT_SUSPENDE@ 0000000180006a50     libiterreachobj001.obj
 0002:00000a78       ??_C@_0BN@FABOLPBI@JVMTI_ERROR_THREAD_SUSPENDED@ 0000000180006a78     libiterreachobj001.obj
 0002:00000a98       ??_C@_0BN@FDGNOBJM@JVMTI_ERROR_THREAD_NOT_ALIVE@ 0000000180006a98     libiterreachobj001.obj
 0002:00000ab8       ??_C@_0BL@GOBIFKNJ@JVMTI_ERROR_INVALID_OBJECT@ 0000000180006ab8     libiterreachobj001.obj
 0002:00000ad8       ??_C@_0BK@FCMAJPPC@JVMTI_ERROR_INVALID_CLASS@ 0000000180006ad8     libiterreachobj001.obj
 0002:00000af8       ??_C@_0BP@IKLLBKEB@JVMTI_ERROR_CLASS_NOT_PREPARED@ 0000000180006af8     libiterreachobj001.obj
 0002:00000b18       ??_C@_0BN@KLPPLKG@JVMTI_ERROR_INVALID_METHODID@ 0000000180006b18     libiterreachobj001.obj
 0002:00000b38       ??_C@_0BN@BCEKOKND@JVMTI_ERROR_INVALID_LOCATION@ 0000000180006b38     libiterreachobj001.obj
 0002:00000b58       ??_C@_0BM@DFDGPME@JVMTI_ERROR_INVALID_FIELDID@ 0000000180006b58     libiterreachobj001.obj
 0002:00000b78       ??_C@_0BL@NELIEPEC@JVMTI_ERROR_NO_MORE_FRAMES@ 0000000180006b78     libiterreachobj001.obj
 0002:00000b98       ??_C@_0BJ@BDBECFDM@JVMTI_ERROR_OPAQUE_FRAME@ 0000000180006b98     libiterreachobj001.obj
 0002:00000bb8       ??_C@_0BK@MIIFNLOB@JVMTI_ERROR_TYPE_MISMATCH@ 0000000180006bb8     libiterreachobj001.obj
 0002:00000bd8       ??_C@_0BJ@HPCAOILC@JVMTI_ERROR_INVALID_SLOT@ 0000000180006bd8     libiterreachobj001.obj
 0002:00000bf8       ??_C@_0BG@CHILOPNI@JVMTI_ERROR_DUPLICATE@ 0000000180006bf8     libiterreachobj001.obj
 0002:00000c10       ??_C@_0BG@DIEMLHKM@JVMTI_ERROR_NOT_FOUND@ 0000000180006c10     libiterreachobj001.obj
 0002:00000c28       ??_C@_0BM@NHMCKHOB@JVMTI_ERROR_INVALID_MONITOR@ 0000000180006c28     libiterreachobj001.obj
 0002:00000c48       ??_C@_0BO@PPEDAJGL@JVMTI_ERROR_NOT_MONITOR_OWNER@ 0000000180006c48     libiterreachobj001.obj
 0002:00000c68       ??_C@_0BG@FCAIPEID@JVMTI_ERROR_INTERRUPT@ 0000000180006c68     libiterreachobj001.obj
 0002:00000c80       ??_C@_0CB@EGDBNKOI@JVMTI_ERROR_INVALID_CLASS_FORMA@ 0000000180006c80     libiterreachobj001.obj
 0002:00000ca8       ??_C@_0CG@DGKOGIAL@JVMTI_ERROR_CIRCULAR_CLASS_DEFI@ 0000000180006ca8     libiterreachobj001.obj
 0002:00000cd0       ??_C@_0BP@ICEALPKC@JVMTI_ERROR_FAILS_VERIFICATION@ 0000000180006cd0     libiterreachobj001.obj
 0002:00000cf0       ??_C@_0DC@JDACLMIO@JVMTI_ERROR_UNSUPPORTED_REDEFIN@ 0000000180006cf0     libiterreachobj001.obj
 0002:00000d28       ??_C@_0DE@GKDKNOMJ@JVMTI_ERROR_UNSUPPORTED_REDEFIN@ 0000000180006d28     libiterreachobj001.obj
 0002:00000d60       ??_C@_0BO@LAFKIOG@JVMTI_ERROR_INVALID_TYPESTATE@ 0000000180006d60     libiterreachobj001.obj
 0002:00000d80       ??_C@_0DH@INDGCLLB@JVMTI_ERROR_UNSUPPORTED_REDEFIN@ 0000000180006d80     libiterreachobj001.obj
 0002:00000db8       ??_C@_0DE@NHEOMMGI@JVMTI_ERROR_UNSUPPORTED_REDEFIN@ 0000000180006db8     libiterreachobj001.obj
 0002:00000df0       ??_C@_0CA@EKPNJOEP@JVMTI_ERROR_UNSUPPORTED_VERSION@ 0000000180006df0     libiterreachobj001.obj
 0002:00000e10       ??_C@_0BN@OFFMAHHL@JVMTI_ERROR_NAMES_DONT_MATCH@ 0000000180006e10     libiterreachobj001.obj
 0002:00000e30       ??_C@_0DN@HHBBLAKE@JVMTI_ERROR_UNSUPPORTED_REDEFIN@ 0000000180006e30     libiterreachobj001.obj
 0002:00000e70       ??_C@_0DO@HMBGBGNA@JVMTI_ERROR_UNSUPPORTED_REDEFIN@ 0000000180006e70     libiterreachobj001.obj
 0002:00000eb0       ??_C@_0BP@PBECGKHJ@JVMTI_ERROR_UNMODIFIABLE_CLASS@ 0000000180006eb0     libiterreachobj001.obj
 0002:00000ed0       ??_C@_0BK@CANILEHF@JVMTI_ERROR_NOT_AVAILABLE@ 0000000180006ed0     libiterreachobj001.obj
 0002:00000ef0       ??_C@_0CE@INJKMEFK@JVMTI_ERROR_MUST_POSSESS_CAPABI@ 0000000180006ef0     libiterreachobj001.obj
 0002:00000f18       ??_C@_0BJ@LBFPFPDM@JVMTI_ERROR_NULL_POINTER@ 0000000180006f18     libiterreachobj001.obj
 0002:00000f38       ??_C@_0BP@CHJPNNEM@JVMTI_ERROR_ABSENT_INFORMATION@ 0000000180006f38     libiterreachobj001.obj
 0002:00000f58       ??_C@_0BP@OMFMNLC@JVMTI_ERROR_INVALID_EVENT_TYPE@ 0000000180006f58     libiterreachobj001.obj
 0002:00000f78       ??_C@_0BN@BIBNPHHO@JVMTI_ERROR_ILLEGAL_ARGUMENT@ 0000000180006f78     libiterreachobj001.obj
 0002:00000f98       ??_C@_0BK@KKNDHDCE@JVMTI_ERROR_NATIVE_METHOD@ 0000000180006f98     libiterreachobj001.obj
 0002:00000fb8       ??_C@_0BK@PMKCFHAE@JVMTI_ERROR_OUT_OF_MEMORY@ 0000000180006fb8     libiterreachobj001.obj
 0002:00000fd8       ??_C@_0BK@NNJBDMNB@JVMTI_ERROR_ACCESS_DENIED@ 0000000180006fd8     libiterreachobj001.obj
 0002:00000ff8       ??_C@_0BI@GHECLMNC@JVMTI_ERROR_WRONG_PHASE@ 0000000180006ff8     libiterreachobj001.obj
 0002:00001010       ??_C@_0BF@OLIHJOII@JVMTI_ERROR_INTERNAL@ 0000000180007010     libiterreachobj001.obj
 0002:00001028       ??_C@_0BO@EOHGKJHI@JVMTI_ERROR_UNATTACHED_THREAD@ 0000000180007028     libiterreachobj001.obj
 0002:00001048       ??_C@_0CA@LKHFDACL@JVMTI_ERROR_INVALID_ENVIRONMENT@ 0000000180007048     libiterreachobj001.obj
 0002:00001068       ??_C@_0BA@MMFHLOKK@?$DMunknown?5error?$DO@ 0000000180007068     libiterreachobj001.obj
 0002:00001078       ??_C@_0CF@CBHOKDB@throwable?5?$DN?5jni?9?$DOExceptionOccur@ 0000000180007078     libiterreachobj001.obj
 0002:000010a0       ??_C@_03OFAPEBGM@?$CFs?6@  00000001800070a0     libiterreachobj001.obj
 0002:000010a8       ??_C@_0DM@LPIGEGNJ@s?2test?2hotspot?2jtreg?2vmTestbase@ 00000001800070a8     libiterreachobj001.obj
 0002:000010e8       ??_C@_0CC@NFCNPEPK@Exception?5in?5JNI?5call?5?$CIcleared?$CJ@ 00000001800070e8     libiterreachobj001.obj
 0002:00001110       ??_C@_0BJ@IBAKFIKF@jni?9?$DOExceptionDescribe?$CI?$CJ@ 0000000180007110     libiterreachobj001.obj
 0002:00001130       ??_C@_0BG@GGKALKMH@jni?9?$DOExceptionClear?$CI?$CJ@ 0000000180007130     libiterreachobj001.obj
 0002:00001148       ??_C@_0CF@JMGFGJLJ@?$CD?5?5?5verified?5JNI?5assertion?5is?5F@ 0000000180007148     libiterreachobj001.obj
 0002:00001170       ??_C@_07KBAMPNJK@verbose@  0000000180007170     libiterreachobj001.obj
 0002:00001178       ??_C@_0DN@PKJBOLAP@nsk_jvmti_parseOptions?$CI?$CJ?3?5unexp@ 0000000180007178     libiterreachobj001.obj
 0002:000011b8       ??_C@_05IMBNNINJ@trace@    00000001800071b8     libiterreachobj001.obj
 0002:000011c0       ??_C@_0DD@BJKGNDMB@nsk_jvmti_parseOptions?$CI?$CJ?3?5no?5va@ 00000001800071c0     libiterreachobj001.obj
 0002:000011f4       ??_C@_04CGFJFPFD@none@     00000001800071f4     libiterreachobj001.obj
 0002:000011fc       ??_C@_06BMELKFMA@before@   00000001800071fc     libiterreachobj001.obj
 0002:00001204       ??_C@_05CMKPCFDK@after@    0000000180007204     libiterreachobj001.obj
 0002:0000120c       ??_C@_03NFKEKGGK@all@      000000018000720c     libiterreachobj001.obj
 0002:00001210       ??_C@_0DM@NDNJGJKE@nsk_jvmti_parseOptions?$CI?$CJ?3?5uexpe@ 0000000180007210     libiterreachobj001.obj
 0002:00001250       ??_C@_08NBBJKJO@waittime@  0000000180007250     libiterreachobj001.obj
 0002:00001260       ??_C@_0DO@CMHGAOHC@nsk_jvmti_parseOptions?$CI?$CJ?3?5not?5i@ 0000000180007260     libiterreachobj001.obj
 0002:000012a0       ??_C@_0DL@LNMPBDLN@nsk_jvmti_parseOptions?$CI?$CJ?3?5negat@ 00000001800072a0     libiterreachobj001.obj
 0002:000012e0       ??_C@_0DA@GMFJNOJH@nsk_jvmti_parseOptions?$CI?$CJ?3?5unkno@ 00000001800072e0     libiterreachobj001.obj
 0002:00001310       ??_C@_0CO@CCIAMEAN@nsk_jvmti_parseOptions?$CI?$CJ?3?5found@ 0000000180007310     libiterreachobj001.obj
 0002:00001340       ??_C@_0CJ@OEGPCGDL@nsk_jvmti_parseOptions?$CI?$CJ?3?5out?5o@ 0000000180007340     libiterreachobj001.obj
 0002:00001370       ??_C@_0DI@NMBHPGGF@nsk_jvmti_parseOptions?$CI?$CJ?3?5too?5m@ 0000000180007370     libiterreachobj001.obj
 0002:000013a8       ??_C@_03POGCGECB@?5?0?$HO@ 00000001800073a8     libiterreachobj001.obj
 0002:000013b0       ??_C@_0DC@GKLNPJIJ@nsk_jvmti_findOptionValue?$CI?$CJ?3?5op@ 00000001800073b0     libiterreachobj001.obj
 0002:000013e8       ??_C@_0DF@OPPIHBPJ@nsk_jvmti_findOptionIntValue?$CI?$CJ?3@ 00000001800073e8     libiterreachobj001.obj
 0002:00001420       ??_C@_0DO@DBKDODPI@nsk_jvmti_findOptionIntValue?$CI?$CJ?3@ 0000000180007420     libiterreachobj001.obj
 0002:00001460       ??_C@_0EE@NGNPKOJC@nsk_jvmti_findOptionIntValue?$CI?$CJ?3@ 0000000180007460     libiterreachobj001.obj
 0002:000014a8       ??_C@_0CB@MLNJNCLJ@?5?5jvmti?5error?3?5code?$DN?$CFd?0?5name?$DN?$CFs@ 00000001800074a8     libiterreachobj001.obj
 0002:000014d0       ??_C@_0CD@OHBGDKMK@?$CD?5?5?5jvmti?5error?3?5code?$DN?$CFd?0?5name?$DN@ 00000001800074d0     libiterreachobj001.obj
 0002:000014f8       ??_C@_0CG@JNNCGPHB@?$CD?5?5?5error?5expected?3?5code?$DN?$CFd?0?5na@ 00000001800074f8     libiterreachobj001.obj
 0002:00001520       ??_C@_0EB@IMGKPCGE@?$CIstr_obj?5?$DN?5jni?9?$DONewStringUTF?$CIco@ 0000000180007520     libiterreachobj001.obj
 0002:00001570       ??_C@_0EA@HFOGGBCC@s?2test?2hotspot?2jtreg?2vmTestbase@ 0000000180007570     libiterreachobj001.obj
 0002:000015b0       ??_C@_05KKCIMGE@error@     00000001800075b0     libiterreachobj001.obj
 0002:000015b8       ??_C@_0CJ@JACLEAA@Test?5failed?5by?5setFailStatus?$CI?$CJ?4@ 00000001800075b8     libiterreachobj001.obj
 0002:000015e8       ??_C@_0BD@HGNAOMCP@agent_data_monitor@ 00000001800075e8     libiterreachobj001.obj
 0002:00001600       ??_C@_0EB@OGCLGKLN@javaVM?9?$DOGetEnv?$CI?$CIvoid?5?$CK?$CK?$CJ?$CGjvmti_@ 0000000180007600     libiterreachobj001.obj
 0002:00001650       ??_C@_0EA@PNBCDMOA@s?2test?2hotspot?2jtreg?2vmTestbase@ 0000000180007650     libiterreachobj001.obj
 0002:00001690       ??_C@_0CI@DDPIFBGM@init_agent_data?$CIjvmti_env?0?5?$CGage@ 0000000180007690     libiterreachobj001.obj
 0002:000016b8       ??_C@_0DI@ILAHDLMP@?$CI?$CKagentThreadProc?$CJ?$CIjvmti_env?0?5a@ 00000001800076b8     libiterreachobj001.obj
 0002:000016f0       ??_C@_0BD@KDBALNLB@JVMTI?5agent?5thread@ 00000001800076f0     libiterreachobj001.obj
 0002:00001708       ??_C@_0BB@NOKBFPFO@java?1lang?1Thread@ 0000000180007708     libiterreachobj001.obj
 0002:0000171c       ??_C@_06FALKBLGB@?$DMinit?$DO@ 000000018000771c     libiterreachobj001.obj
 0002:00001728       ??_C@_0BG@IKDDPPGD@?$CILjava?1lang?1String?$DL?$CJV@ 0000000180007728     libiterreachobj001.obj
 0002:00001740       ??_C@_0EB@IFJBFEKC@?$CIthreadClass?5?$DN?5jni_env?9?$DOFindCla@ 0000000180007740     libiterreachobj001.obj
 0002:00001790       ??_C@_0GF@FGFIBKKL@?$CIthreadCtor?5?$DN?5jni_env?9?$DOGetMetho@ 0000000180007790     libiterreachobj001.obj
 0002:000017f8       ??_C@_0DN@NCPDJLOG@?$CIthreadName?5?$DN?5jni_env?9?$DONewStrin@ 00000001800077f8     libiterreachobj001.obj
 0002:00001840       ??_C@_0FE@PFKODBGC@?$CIthreadObject?5?$DN?5jni_env?9?$DONewObj@ 0000000180007840     libiterreachobj001.obj
 0002:000018a0       ??_C@_0ED@HOBAHHJI@?$CIthreadGlobalRef?5?$DN?5jni_env?9?$DONew@ 00000001800078a0     libiterreachobj001.obj
 0002:000018f0       ??_C@_0FN@HNJJAHFC@jvmti_env?9?$DORunAgentThread?$CIagent@ 00000001800078f0     libiterreachobj001.obj
 0002:00001950       ??_C@_0EA@MOJDNKDF@Debuggee?5status?5sync?5aborted?5be@ 0000000180007950     libiterreachobj001.obj
 0002:00001990       ??_C@_0CO@PGPGMHBJ@No?5status?5sync?5occured?5for?5time@ 0000000180007990     libiterreachobj001.obj
 0002:000019c0       ??_C@_0CL@DOEBDPKJ@Debuggee?5was?5not?5suspended?5on?5s@ 00000001800079c0     libiterreachobj001.obj
 0002:000019f0       ??_C@_0EA@EEOEJAEN@status?5?$DN?5syncDebuggeeStatus?$CIjni@ 00000001800079f0     libiterreachobj001.obj
 0002:00001a30       ??_C@_0BL@JBCFNBMB@nsk_jvmti_resetAgentData?$CI?$CJ@ 0000000180007a30     libiterreachobj001.obj
 0002:00001a50       ??_C@_0EL@LPBEELIP@s?2test?2hotspot?2jtreg?2vmTestbase@ 0000000180007a50     libiterreachobj001.obj
 0002:00001aa0       ??_C@_0CK@JDAMFDMJ@jvmti?9?$DOSetTag?$CIo?0?5tag?$CJ?5?$DN?$DN?5JVMTI_@ 0000000180007aa0     libiterreachobj001.obj
 0002:00001ad0       ??_C@_0CC@DAMNHKNI@Can?8t?5set?5tag?5?$CFli?5for?5object?5?$CFl@ 0000000180007ad0     libiterreachobj001.obj
 0002:00001af8       ??_C@_0DL@HAJPNKEF@jvmti?9?$DOGetObjectHashCode?$CIo?0?5?$CGha@ 0000000180007af8     libiterreachobj001.obj
 0002:00001b38       ??_C@_0BL@JFPIEOBF@Can?8t?5get?5hash?5object?5?$CFlx?6@ 0000000180007b38     libiterreachobj001.obj
 0002:00001b58       ??_C@_0BG@DICPHBKN@setTag?3?5?$CF08x?5?$DM?9?5?$CF?53li@ 0000000180007b58     libiterreachobj001.obj
 0002:00001b70       ??_C@_0DH@FCEEBDMJ@?$CIs?5?$DN?5jni?9?$DOGetStringUTFChars?$CIsIn@ 0000000180007b70     libiterreachobj001.obj
 0002:00001ba8       ??_C@_0BJ@OKKGHDCN@Can?8t?5get?5string?5at?5?$CF?$CDp?6@ 0000000180007ba8     libiterreachobj001.obj
 0002:00001bc8       ??_C@_0BP@EKFLGGFJ@Can?8t?5get?5string?5at?5?$CF?$CDp?3?5null?6@ 0000000180007bc8     libiterreachobj001.obj
 0002:00001be8       ??_C@_06ICODBHCL@?5?1?1?5?$CFs@ 0000000180007be8     libiterreachobj001.obj
 0002:00001bf0       ??_C@_0DB@KGFPLEGO@?$CIr?5?$DN?5jvmti?9?$DOGetTag?$CIo?0?5?$CGtag?$CJ?$CJ?5?$DN?$DN@ 0000000180007bf0     libiterreachobj001.obj
 0002:00001c28       ??_C@_0CO@PDAGBCGJ@Can?8t?5GetTag?5for?5object?5?$CFlx?4?5Re@ 0000000180007c28     libiterreachobj001.obj
 0002:00001c58       ??_C@_0CH@HPEODOHC@TEST_BUG?3?5Max?4?5number?5of?5refs?5r@ 0000000180007c58     libiterreachobj001.obj
 0002:00001c80       ??_C@_0DI@PHFCABIM@?$CIr?5?$DN?5jvmti?9?$DOGetTag?$CIfrom?0?5?$CGtagFr@ 0000000180007c80     libiterreachobj001.obj
 0002:00001cb8       ??_C@_0DI@MDEGFNKD@TEST_BUG?3?5Can?8t?5GetTag?5for?5obje@ 0000000180007cb8     libiterreachobj001.obj
 0002:00001cf0       ??_C@_0DE@MLELJAHM@?$CIr?5?$DN?5jvmti?9?$DOGetTag?$CIto?0?5?$CGtagTo?$CJ?$CJ@ 0000000180007cf0     libiterreachobj001.obj
 0002:00001d30       ??_C@_0EA@OLCLFBLL@?$CIobj?5?$DN?5jni?9?$DOGetObjectField?$CIfirs@ 0000000180007d30     libiterreachobj001.obj
 0002:00001d70       ??_C@_0GK@EIACOHPC@s?2test?2hotspot?2jtreg?2vmTestbase@ 0000000180007d70     libiterreachobj001.obj
 0002:00001de0       ??_C@_0BL@HDOCIPLI@jvmti?9?$DOSetTag?$CIobj?0?5objTag?$CJ@ 0000000180007de0     libiterreachobj001.obj
 0002:00001e00       ??_C@_0BP@KLIOMM@?5?5?5?5?5?5?5?5tag?$DN?$CF?95ld?5object?$DN0x?$CFp?6@ 0000000180007e00     libiterreachobj001.obj
 0002:00001e20       ??_C@_0BJ@NBEMCAEP@jni?9?$DODeleteLocalRef?$CIobj?$CJ@ 0000000180007e20     libiterreachobj001.obj
 0002:00001e40       ??_C@_0CO@OFDFJEOH@Allocate?5memory?5for?5objects?5lis@ 0000000180007e40     libiterreachobj001.obj
 0002:00001e70       ??_C@_0FH@KENAHJKN@jvmti?9?$DOAllocate?$CI?$CI?$CKobjectsCount?5@ 0000000180007e70     libiterreachobj001.obj
 0002:00001ec8       ??_C@_0BN@GHDOCCDB@?5?5?4?4?4?5allocated?5array?3?50x?$CFp?6@ 0000000180007ec8     libiterreachobj001.obj
 0002:00001ee8       ??_C@_0DG@CKHACGKM@nsk?1jvmti?1IterateOverReachableO@ 0000000180007ee8     libiterreachobj001.obj
 0002:00001f20       ??_C@_0BI@ENEOJHP@Find?5debugee?5class?3?5?$CFs?6@ 0000000180007f20     libiterreachobj001.obj
 0002:00001f38       ??_C@_0DP@MFMMLPOM@?$CIdebugeeClass?5?$DN?5jni?9?$DOFindClass?$CI@ 0000000180007f38     libiterreachobj001.obj
 0002:00001f78       ??_C@_0BJ@DFGCANJI@?5?5?4?4?4?5found?5class?3?50x?$CFp?6@ 0000000180007f78     libiterreachobj001.obj
 0002:00001fa0       ??_C@_0EF@EKKEOCLA@nsk?1jvmti?1IterateOverReachableO@ 0000000180007fa0     libiterreachobj001.obj
 0002:00001fe8       ??_C@_0BM@GFHMIOD@Find?5root?5object?5class?3?5?$CFs?6@ 0000000180007fe8     libiterreachobj001.obj
 0002:00002010       ??_C@_0EG@LBKAPJFG@?$CIrootObjectClass?5?$DN?5jni?9?$DOFindCla@ 0000000180008010     libiterreachobj001.obj
 0002:00002060       ??_C@_0EB@GMDNFJOF@nsk?1jvmti?1IterateOverReachableO@ 0000000180008060     libiterreachobj001.obj
 0002:000020a8       ??_C@_0BN@JPFPOKGN@Find?5chain?5object?5class?3?5?$CFs?6@ 00000001800080a8     libiterreachobj001.obj
 0002:000020d0       ??_C@_0EI@PFABFCAO@?$CIchainObjectClass?5?$DN?5jni?9?$DOFindCl@ 00000001800080d0     libiterreachobj001.obj
 0002:00002118       ??_C@_06IEOJBDIK@object@   0000000180008118     libiterreachobj001.obj
 0002:00002120       ??_C@_0CI@IPDCJCKO@Find?5static?5field?5in?5debugee?5cl@ 0000000180008120     libiterreachobj001.obj
 0002:00002150       ??_C@_0GK@JEMGECFG@?$CIobjectField?5?$DN?5jni?9?$DOGetStaticFi@ 0000000180008150     libiterreachobj001.obj
 0002:000021c0       ??_C@_0EH@POIILBGH@Lnsk?1jvmti?1IterateOverReachable@ 00000001800081c0     libiterreachobj001.obj
 0002:00002208       ??_C@_0BJ@MIIADDIH@?5?5?4?4?4?5got?5fieldID?3?50x?$CFp?6@ 0000000180008208     libiterreachobj001.obj
 0002:00002228       ??_C@_0P@OFCAMOEL@reachableChain@ 0000000180008228     libiterreachobj001.obj
 0002:00002238       ??_C@_0CO@GJFDOONJ@Find?5instance?5field?5in?5root?5obj@ 0000000180008238     libiterreachobj001.obj
 0002:00002270       ??_C@_0HJ@BDIDKFJF@?$CIreachableChainField?5?$DN?5jni?9?$DOGet@ 0000000180008270     libiterreachobj001.obj
 0002:000022f0       ??_C@_0ED@JCBNIANN@Lnsk?1jvmti?1IterateOverReachable@ 00000001800082f0     libiterreachobj001.obj
 0002:00002338       ??_C@_0BB@HCMFGFMC@unreachableChain@ 0000000180008338     libiterreachobj001.obj
 0002:00002350       ??_C@_0HN@KPAGODBH@?$CIunreachableChainField?5?$DN?5jni?9?$DOG@ 0000000180008350     libiterreachobj001.obj
 0002:000023d0       ??_C@_04DIFLAKIP@tail@     00000001800083d0     libiterreachobj001.obj
 0002:000023d8       ??_C@_0CP@FJDMDHPJ@Find?5instance?5field?5in?5chain?5ob@ 00000001800083d8     libiterreachobj001.obj
 0002:00002410       ??_C@_0GE@BFDKKHME@?$CItailField?5?$DN?5jni?9?$DOGetFieldID?$CIch@ 0000000180008410     libiterreachobj001.obj
 0002:00002478       ??_C@_0CH@IEEMMCJA@Get?5root?5object?5from?5static?5fie@ 0000000180008478     libiterreachobj001.obj
 0002:000024a0       ??_C@_0EP@FMMDHOMP@?$CIrootObject?5?$DN?5jni?9?$DOGetStaticObj@ 00000001800084a0     libiterreachobj001.obj
 0002:000024f0       ??_C@_0BI@FNLCMIKO@?5?5?4?4?4?5got?5object?3?50x?$CFp?6@ 00000001800084f0     libiterreachobj001.obj
 0002:00002508       ??_C@_0BP@MAGAMBHE@Obtain?5and?5tag?5chain?5objects?3?6@ 0000000180008508     libiterreachobj001.obj
 0002:00002528       ??_C@_0CJ@ELCOJLPK@?5?5?5?5reachable?5objects?5chain?3?5?$CFd@ 0000000180008528     libiterreachobj001.obj
 0002:00002558       ??_C@_0CL@LBFMJNLN@?5?5?5?5unreachable?5objects?5chain?3?5@ 0000000180008558     libiterreachobj001.obj
 0002:00002588       ??_C@_0CJ@OGMDHCIM@Following?5tagged?5objects?5were?5i@ 0000000180008588     libiterreachobj001.obj
 0002:000025b8       ??_C@_0BI@FLMBJNKJ@?5?5?5?5reachable?5objects?3?6@ 00000001800085b8     libiterreachobj001.obj
 0002:000025d0       ??_C@_0CC@OEHLDPCF@?5?5?5?5?5?5?5?5tag?$DN?$CF?95ld?5found?$DN?$CFd?5time@ 00000001800085d0     libiterreachobj001.obj
 0002:00002600       ??_C@_0EN@LHMMAOGM@Reachable?5object?5was?5not?5iterat@ 0000000180008600     libiterreachobj001.obj
 0002:00002650       ??_C@_0BK@GHAJMINB@?5?5?5?5unreachable?5objects?3?6@ 0000000180008650     libiterreachobj001.obj
 0002:00002670       ??_C@_0EL@NFIOLHMC@Unreachable?5object?5was?5iterated@ 0000000180008670     libiterreachobj001.obj
 0002:000026c0       ??_C@_0BP@JPEMGJLC@Deallocate?5objects?5list?3?50x?$CFp?6@ 00000001800086c0     libiterreachobj001.obj
 0002:000026e0       ??_C@_0DC@DFJJAFOM@jvmti?9?$DODeallocate?$CI?$CIunsigned?5cha@ 00000001800086e0     libiterreachobj001.obj
 0002:00002720       ??_C@_0EN@HKALEDNF@?5?5heapRootCallback?3?5root_kind?$DN?$CF@ 0000000180008720     libiterreachobj001.obj
 0002:00002770       ??_C@_0IN@GDDABHLD@null?5tag_ptr?5is?5passed?5to?5heapR@ 0000000180008770     libiterreachobj001.obj
 0002:00002800       ??_C@_0JG@MOOPHFND@Unreachable?5tagged?5object?5passe@ 0000000180008800     libiterreachobj001.obj
 0002:000028a0       ??_C@_0JN@IECDIPGA@Not?5root?5reachable?5tagged?5objec@ 00000001800088a0     libiterreachobj001.obj
 0002:00002940       ??_C@_0JC@PEKFPJHB@Unknown?5tagged?5object?5passed?5to@ 0000000180008940     libiterreachobj001.obj
 0002:000029e0       ??_C@_0GH@CPJALONA@Unexpected?5user_data?5is?5passed?5@ 00000001800089e0     libiterreachobj001.obj
 0002:00002a50       ??_C@_0IC@EBOIGCHA@?5?5stackReferenceCallback?3?5root_@ 0000000180008a50     libiterreachobj001.obj
 0002:00002ae0       ??_C@_0PC@GIJNNLM@null?5tag_ptr?5is?5passed?5to?5stack@ 0000000180008ae0     libiterreachobj001.obj
 0002:00002be0       ??_C@_0PL@JNHKIIEI@Unreachable?5tagged?5object?5passe@ 0000000180008be0     libiterreachobj001.obj
 0002:00002ce0       ??_C@_0BAD@BOMGHAPF@Not?5stack?5reachable?5tagged?5obje@ 0000000180008ce0     libiterreachobj001.obj
 0002:00002df0       ??_C@_0PH@FFNMBGGD@Unknown?5tagged?5object?5passed?5to@ 0000000180008df0     libiterreachobj001.obj
 0002:00002ef0       ??_C@_0GN@BFEEPHJI@Unexpected?5user_data?5is?5passed?5@ 0000000180008ef0     libiterreachobj001.obj
 0002:00002f60       ??_C@_0GM@GIAGPDJJ@?5?5objectReferenceCallback?3?5ref_@ 0000000180008f60     libiterreachobj001.obj
 0002:00002fd0       ??_C@_0MD@KMLMJEHE@null?5tag_ptr?5is?5passed?5to?5objec@ 0000000180008fd0     libiterreachobj001.obj
 0002:000030a0       ??_C@_0MP@DGJCBEAJ@Unreachable?5tagged?5object?5is?5pa@ 00000001800090a0     libiterreachobj001.obj
 0002:00003170       ??_C@_0ML@GPPDEJEA@Unknown?5tagged?5object?5is?5passed@ 0000000180009170     libiterreachobj001.obj
 0002:00003240       ??_C@_0GO@MEKABAMN@Unexpected?5user_data?5is?5passed?5@ 0000000180009240     libiterreachobj001.obj
 0002:000032b0       ??_C@_0CB@KHPCBPAO@Wait?5for?5tested?5objects?5created@ 00000001800092b0     libiterreachobj001.obj
 0002:000032d8       ??_C@_0BP@LAIJOMPC@nsk_jvmti_waitForSync?$CItimeout?$CJ@ 00000001800092d8     libiterreachobj001.obj
 0002:000032f8       ??_C@_0DG@CILGJCLA@?$DO?$DO?$DO?5Obtain?5and?5tag?5tested?5objec@ 00000001800092f8     libiterreachobj001.obj
 0002:00003330       ??_C@_0EK@JHAEBCIG@getTestedObjects?$CIjvmti?0?5jni?0?5ch@ 0000000180009330     libiterreachobj001.obj
 0002:00003380       ??_C@_0DH@PBGGKADM@?$DO?$DO?$DO?5Let?5debugee?5to?5clean?5links?5@ 0000000180009380     libiterreachobj001.obj
 0002:000033b8       ??_C@_0BH@LECMGIIA@nsk_jvmti_resumeSync?$CI?$CJ@ 00000001800093b8     libiterreachobj001.obj
 0002:000033d0       ??_C@_0CM@BFIFLFFB@?$DO?$DO?$DO?5Start?5iteration?5over?5reacha@ 00000001800093d0     libiterreachobj001.obj
 0002:00003400       ??_C@_0HF@PMKMAAJI@jvmti?9?$DOIterateOverReachableObje@ 0000000180009400     libiterreachobj001.obj
 0002:00003478       ??_C@_0CP@KBDHMAKH@?$DO?$DO?$DO?5Check?5if?5reachable?5objects?5@ 0000000180009478     libiterreachobj001.obj
 0002:000034a8       ??_C@_0BF@MNKEFEOE@?$DO?$DO?$DO?5Clean?5used?5data?6@ 00000001800094a8     libiterreachobj001.obj
 0002:000034c0       ??_C@_0DO@OPFNMOBD@releaseTestedObjects?$CIjvmti?0?5jni@ 00000001800094c0     libiterreachobj001.obj
 0002:00003500       ??_C@_0BH@HPEOJMHL@Let?5debugee?5to?5finish?6@ 0000000180009500     libiterreachobj001.obj
 0002:00003518       ??_C@_0CA@MNKGCBCG@nsk_jvmti_parseOptions?$CIoptions?$CJ@ 0000000180009518     libiterreachobj001.obj
 0002:00003538       ??_C@_04NIDJFNBE@info@     0000000180009538     libiterreachobj001.obj
 0002:00003540       ??_C@_06DFFOHAMN@objref@   0000000180009540     libiterreachobj001.obj
 0002:00003548       ??_C@_08JAMFKCP@stackref@  0000000180009548     libiterreachobj001.obj
 0002:00003558       ??_C@_08KICKEILH@heaproot@ 0000000180009558     libiterreachobj001.obj
 0002:00003568       ??_C@_07MNCDLPNM@heapobj@  0000000180009568     libiterreachobj001.obj
 0002:00003570       ??_C@_0BP@PNAOMHNJ@Unknown?5option?5value?3?5info?$DN?$CFs?6@ 0000000180009570     libiterreachobj001.obj
 0002:00003590       ??_C@_07JPLKJBI@objects@   0000000180009590     libiterreachobj001.obj
 0002:00003598       ??_C@_0BA@LIAABLEG@chainLength?5?$DO?50@ 0000000180009598     libiterreachobj001.obj
 0002:000035a8       ??_C@_0DN@MIAMNFPH@?$CIjvmti?5?$DN?5nsk_jvmti_createJVMTIE@ 00000001800095a8     libiterreachobj001.obj
 0002:000035e8       ??_C@_0BO@DBKDIPGD@jvmti?9?$DOAddCapabilities?$CI?$CGcaps?$CJ@ 00000001800095e8     libiterreachobj001.obj
 0002:00003608       ??_C@_0CL@PIACJIPK@nsk_jvmti_setAgentProc?$CIagentPro@ 0000000180009608     libiterreachobj001.obj
 0002:00003650       ??_C@_1EC@JIJBPKFM@?$AAa?$AAp?$AAi?$AA?9?$AAm?$AAs?$AA?9?$AAw?$AAi?$AAn?$AA?9?$AAc?$AAo?$AAr?$AAe@ 0000000180009650     MSVCRT:thread_safe_statics.obj
 0002:00003698       ??_C@_1BK@MGMFAEKH@?$AAk?$AAe?$AAr?$AAn?$AAe?$AAl?$AA3?$AA2?$AA?4?$AAd?$AAl?$AAl@ 0000000180009698     MSVCRT:thread_safe_statics.obj
 0002:000036b8       ??_C@_0BJ@JEBJOJFJ@SleepConditionVariableCS@ 00000001800096b8     MSVCRT:thread_safe_statics.obj
 0002:000036d8       ??_C@_0BJ@PGPPEPCC@WakeAllConditionVariable@ 00000001800096d8     MSVCRT:thread_safe_statics.obj
 0002:000036f8       _pDefaultRawDllMain        00000001800096f8     MSVCRT:dll_dllmain.obj
 0002:000036f8       _pRawDllMain               00000001800096f8     MSVCRT:dll_dllmain.obj
 0002:00003700       __xmm@ffffffffffffffffffffffffffffffff 0000000180009700     MSVCRT:utility.obj
 0002:00003710       _load_config_used          0000000180009710     MSVCRT:loadcfg.obj
 0002:00003900       _tls_used                  0000000180009900     MSVCRT:tlssup.obj
 0002:00003928       __volatile_metadata        0000000180009928     <linker-defined>
 0002:00003d00       __rtc_iaa                  0000000180009d00     MSVCRT:initsect.obj
 0002:00003d08       __rtc_izz                  0000000180009d08     MSVCRT:initsect.obj
 0002:00003d10       __rtc_taa                  0000000180009d10     MSVCRT:initsect.obj
 0002:00003d18       __rtc_tzz                  0000000180009d18     MSVCRT:initsect.obj
 0002:00003d20       _tls_start                 0000000180009d20     MSVCRT:tlssup.obj
 0002:00003d24       _Init_thread_epoch         0000000180009d24     MSVCRT:thread_safe_statics.obj
 0002:00003d28       _tls_end                   0000000180009d28     MSVCRT:tlssup.obj
 0002:00004498       __IMPORT_DESCRIPTOR_KERNEL32 000000018000a498     kernel32:KERNEL32.dll
 0002:000044ac       __IMPORT_DESCRIPTOR_VCRUNTIME140 000000018000a4ac     vcruntime:VCRUNTIME140.dll
 0002:000044c0       __IMPORT_DESCRIPTOR_api-ms-win-crt-heap-l1-1-0 000000018000a4c0     ucrt:api-ms-win-crt-heap-l1-1-0.dll
 0002:000044d4       __IMPORT_DESCRIPTOR_api-ms-win-crt-runtime-l1-1-0 000000018000a4d4     ucrt:api-ms-win-crt-runtime-l1-1-0.dll
 0002:000044e8       __IMPORT_DESCRIPTOR_api-ms-win-crt-convert-l1-1-0 000000018000a4e8     ucrt:api-ms-win-crt-convert-l1-1-0.dll
 0002:000044fc       __IMPORT_DESCRIPTOR_api-ms-win-crt-stdio-l1-1-0 000000018000a4fc     ucrt:api-ms-win-crt-stdio-l1-1-0.dll
 0002:00004510       __IMPORT_DESCRIPTOR_api-ms-win-crt-string-l1-1-0 000000018000a510     ucrt:api-ms-win-crt-string-l1-1-0.dll
 0002:00004524       __NULL_IMPORT_DESCRIPTOR   000000018000a524     kernel32:KERNEL32.dll
 0003:00000030       _Init_global_epoch         000000018000b030     MSVCRT:thread_safe_statics.obj
 0003:00000040       __security_cookie          000000018000b040     MSVCRT:gs_cookie.obj
 0003:00000048       __security_cookie_complement 000000018000b048     MSVCRT:gs_cookie.obj
 0003:00000050       __scrt_native_dllmain_reason 000000018000b050     MSVCRT:utility.obj
 0003:00000058       __isa_available            000000018000b058     MSVCRT:cpu_disp.obj
 0003:0000005c       __isa_enabled              000000018000b05c     MSVCRT:cpu_disp.obj
 0003:00000060       __memset_fast_string_threshold 000000018000b060     MSVCRT:cpu_disp.obj
 0003:00000068       __memset_nt_threshold      000000018000b068     MSVCRT:cpu_disp.obj
 0003:00000070       __scrt_ucrt_dll_is_in_use  000000018000b070     MSVCRT:ucrt_stubs.obj
 0003:00000080       g_wrongHeapCallbacks       000000018000b080     libiterreachobj001.obj
 0003:00000100       g_szTagInfo                000000018000b100     libiterreachobj001.obj
 0003:00002040       g_tagFlags                 000000018000d040     libiterreachobj001.obj
 0003:00002428       g_refsToVerifyCnt          000000018000d428     libiterreachobj001.obj
 0003:0000242c       g_fakeUserData             000000018000d42c     libiterreachobj001.obj
 0003:00002430       g_tagVisitCount            000000018000d430     libiterreachobj001.obj
 0003:000033d0       g_refsToVerify             000000018000e3d0     libiterreachobj001.obj
 0003:0001aad0       g_userDataError            0000000180025ad0     libiterreachobj001.obj
 0003:0001ac88       ?_OptionsStorage@?1??__local_stdio_printf_options@@9@4_KA 0000000180025c88     libiterreachobj001.obj
 0003:0001b248       _tls_index                 0000000180026248     MSVCRT:tlssup.obj
 0003:0001b250       __scrt_current_native_startup_state 0000000180026250     MSVCRT:utility.obj
 0003:0001b258       __scrt_native_startup_lock 0000000180026258     MSVCRT:utility.obj
 0003:0001b298       __scrt_debugger_hook_flag  0000000180026298     MSVCRT:utility_desktop.obj
 0003:0001b2a0       ?__type_info_root_node@@3U__type_info_node@@A 00000001800262a0     MSVCRT:tncleanup.obj
 0003:0001b2b0       ?_OptionsStorage@?1??__local_stdio_scanf_options@@9@4_KA 00000001800262b0     MSVCRT:default_local_stdio_options.obj
 0003:0001b2b8       __favor                    00000001800262b8     MSVCRT:cpu_disp.obj
 0003:0001b2c0       __dyn_tls_init_callback    00000001800262c0     <common>

 entry point at        0001:000041d0

 Static symbols

 0000:fffd7000       .debug$S                   0000000180000000     iterreachobj001.exp
 0000:fffd7000       .debug$S                   0000000180000000     vcruntime:VCRUNTIME140.dll
 0000:fffd7000       .debug$S                   0000000180000000     vcruntime:VCRUNTIME140.dll
 0000:fffd7000       .debug$S                   0000000180000000     vcruntime:VCRUNTIME140.dll
 0000:fffd7000       .debug$S                   0000000180000000     vcruntime:VCRUNTIME140.dll
 0000:fffd7000       .debug$S                   0000000180000000     vcruntime:VCRUNTIME140.dll
 0000:fffd7000       .debug$S                   0000000180000000     vcruntime:VCRUNTIME140.dll
 0000:fffd7000       .debug$S                   0000000180000000     vcruntime:VCRUNTIME140.dll
 0000:fffd7000       .debug$S                   0000000180000000     ucrt:api-ms-win-crt-convert-l1-1-0.dll
 0000:fffd7000       .debug$S                   0000000180000000     ucrt:api-ms-win-crt-heap-l1-1-0.dll
 0000:fffd7000       .debug$S                   0000000180000000     ucrt:api-ms-win-crt-heap-l1-1-0.dll
 0000:fffd7000       .debug$S                   0000000180000000     ucrt:api-ms-win-crt-heap-l1-1-0.dll
 0000:fffd7000       .debug$S                   0000000180000000     ucrt:api-ms-win-crt-heap-l1-1-0.dll
 0000:fffd7000       .debug$S                   0000000180000000     ucrt:api-ms-win-crt-runtime-l1-1-0.dll
 0000:fffd7000       .debug$S                   0000000180000000     ucrt:api-ms-win-crt-runtime-l1-1-0.dll
 0000:fffd7000       .debug$S                   0000000180000000     ucrt:api-ms-win-crt-runtime-l1-1-0.dll
 0000:fffd7000       .debug$S                   0000000180000000     ucrt:api-ms-win-crt-runtime-l1-1-0.dll
 0000:fffd7000       .debug$S                   0000000180000000     ucrt:api-ms-win-crt-runtime-l1-1-0.dll
 0000:fffd7000       .debug$S                   0000000180000000     ucrt:api-ms-win-crt-runtime-l1-1-0.dll
 0000:fffd7000       .debug$S                   0000000180000000     ucrt:api-ms-win-crt-runtime-l1-1-0.dll
 0000:fffd7000       .debug$S                   0000000180000000     ucrt:api-ms-win-crt-runtime-l1-1-0.dll
 0000:fffd7000       .debug$S                   0000000180000000     ucrt:api-ms-win-crt-runtime-l1-1-0.dll
 0000:fffd7000       .debug$S                   0000000180000000     ucrt:api-ms-win-crt-runtime-l1-1-0.dll
 0000:fffd7000       .debug$S                   0000000180000000     ucrt:api-ms-win-crt-runtime-l1-1-0.dll
 0000:fffd7000       .debug$S                   0000000180000000     ucrt:api-ms-win-crt-runtime-l1-1-0.dll
 0000:fffd7000       .debug$S                   0000000180000000     ucrt:api-ms-win-crt-runtime-l1-1-0.dll
 0000:fffd7000       .debug$S                   0000000180000000     ucrt:api-ms-win-crt-runtime-l1-1-0.dll
 0000:fffd7000       .debug$S                   0000000180000000     ucrt:api-ms-win-crt-runtime-l1-1-0.dll
 0000:fffd7000       .debug$S                   0000000180000000     ucrt:api-ms-win-crt-runtime-l1-1-0.dll
 0000:fffd7000       .debug$S                   0000000180000000     ucrt:api-ms-win-crt-stdio-l1-1-0.dll
 0000:fffd7000       .debug$S                   0000000180000000     ucrt:api-ms-win-crt-stdio-l1-1-0.dll
 0000:fffd7000       .debug$S                   0000000180000000     ucrt:api-ms-win-crt-stdio-l1-1-0.dll
 0000:fffd7000       .debug$S                   0000000180000000     ucrt:api-ms-win-crt-stdio-l1-1-0.dll
 0000:fffd7000       .debug$S                   0000000180000000     ucrt:api-ms-win-crt-stdio-l1-1-0.dll
 0000:fffd7000       .debug$S                   0000000180000000     ucrt:api-ms-win-crt-stdio-l1-1-0.dll
 0000:fffd7000       .debug$S                   0000000180000000     ucrt:api-ms-win-crt-stdio-l1-1-0.dll
 0000:fffd7000       .debug$S                   0000000180000000     ucrt:api-ms-win-crt-stdio-l1-1-0.dll
 0000:fffd7000       .debug$S                   0000000180000000     ucrt:api-ms-win-crt-stdio-l1-1-0.dll
 0000:fffd7000       .debug$S                   0000000180000000     ucrt:api-ms-win-crt-stdio-l1-1-0.dll
 0000:fffd7000       .debug$S                   0000000180000000     ucrt:api-ms-win-crt-string-l1-1-0.dll
 0000:fffd7000       .debug$S                   0000000180000000     ucrt:api-ms-win-crt-string-l1-1-0.dll
 0000:fffd7000       .debug$S                   0000000180000000     ucrt:api-ms-win-crt-string-l1-1-0.dll
 0000:fffd7000       .debug$S                   0000000180000000     ucrt:api-ms-win-crt-string-l1-1-0.dll
 0000:fffd7000       .debug$S                   0000000180000000     ucrt:api-ms-win-crt-string-l1-1-0.dll
 0000:fffd7000       .debug$S                   0000000180000000     ucrt:api-ms-win-crt-string-l1-1-0.dll
 0000:fffd7000       .debug$S                   0000000180000000     ucrt:api-ms-win-crt-string-l1-1-0.dll
 0000:fffd7000       .debug$S                   0000000180000000     ucrt:api-ms-win-crt-string-l1-1-0.dll
 0000:fffd7000       .debug$S                   0000000180000000     kernel32:KERNEL32.dll
 0000:fffd7000       .debug$S                   0000000180000000     kernel32:KERNEL32.dll
 0000:fffd7000       .debug$S                   0000000180000000     kernel32:KERNEL32.dll
 0000:fffd7000       .debug$S                   0000000180000000     kernel32:KERNEL32.dll
 0000:fffd7000       .debug$S                   0000000180000000     kernel32:KERNEL32.dll
 0000:fffd7000       .debug$S                   0000000180000000     kernel32:KERNEL32.dll
 0000:fffd7000       .debug$S                   0000000180000000     kernel32:KERNEL32.dll
 0000:fffd7000       .debug$S                   0000000180000000     kernel32:KERNEL32.dll
 0000:fffd7000       .debug$S                   0000000180000000     kernel32:KERNEL32.dll
 0000:fffd7000       .debug$S                   0000000180000000     kernel32:KERNEL32.dll
 0000:fffd7000       .debug$S                   0000000180000000     kernel32:KERNEL32.dll
 0000:fffd7000       .debug$S                   0000000180000000     kernel32:KERNEL32.dll
 0000:fffd7000       .debug$S                   0000000180000000     kernel32:KERNEL32.dll
 0000:fffd7000       .debug$S                   0000000180000000     kernel32:KERNEL32.dll
 0000:fffd7000       .debug$S                   0000000180000000     kernel32:KERNEL32.dll
 0000:fffd7000       .debug$S                   0000000180000000     kernel32:KERNEL32.dll
 0000:fffd7000       .debug$S                   0000000180000000     kernel32:KERNEL32.dll
 0000:fffd7000       .debug$S                   0000000180000000     kernel32:KERNEL32.dll
 0000:fffd7000       .debug$S                   0000000180000000     kernel32:KERNEL32.dll
 0000:fffd7000       .debug$S                   0000000180000000     kernel32:KERNEL32.dll
 0000:fffd7000       .debug$S                   0000000180000000     kernel32:KERNEL32.dll
 0000:fffd7000       .debug$S                   0000000180000000     kernel32:KERNEL32.dll
 0000:fffd7000       .debug$S                   0000000180000000     kernel32:KERNEL32.dll
 0000:fffd7000       .debug$S                   0000000180000000     kernel32:KERNEL32.dll
 0000:fffd7000       .debug$S                   0000000180000000     kernel32:KERNEL32.dll
 0000:fffd7000       .debug$S                   0000000180000000     kernel32:KERNEL32.dll
 0000:fffd7000       .debug$S                   0000000180000000     kernel32:KERNEL32.dll
 0000:fffd7000       .debug$S                   0000000180000000     kernel32:KERNEL32.dll
 0001:00000fa0       addRefToVerify             0000000180001fa0 f   libiterreachobj001.obj
 0001:0000100c       agentProc                  000000018000200c f   libiterreachobj001.obj
 0001:00001384       agentThreadWrapper         0000000180002384 f   libiterreachobj001.obj
 0001:000014f0       checkTestedObjects         00000001800024f0 f   libiterreachobj001.obj
 0001:00001664       check_option               0000000180002664 f   libiterreachobj001.obj
 0001:000018ac       file_basename              00000001800028ac f   libiterreachobj001.obj
 0001:00001920       getChainObjects            0000000180002920 f   libiterreachobj001.obj
 0001:00001b84       getTestedObjects           0000000180002b84 f   libiterreachobj001.obj
 0001:0000339c       releaseTestedObjects       000000018000439c f   libiterreachobj001.obj
 0001:000036b8       startAgentThreadWrapper    00000001800046b8 f   libiterreachobj001.obj
 0001:000039f8       syncDebuggeeStatus         00000001800049f8 f   libiterreachobj001.obj
 0001:00003c98       capture_previous_context   0000000180004c98 f   MSVCRT:gs_report.obj
 0001:00003d0c       ?__scrt_initialize_thread_safe_statics@@YAHXZ 0000000180004d0c f   MSVCRT:thread_safe_statics.obj
 0001:00003ddc       ?__scrt_uninitialize_thread_safe_statics@@YAXXZ 0000000180004ddc f   MSVCRT:thread_safe_statics.obj
 0001:00003e80       $$000000                   0000000180004e80     MSVCRT:amdsecgs.obj
 0001:00003eb0       ?dllmain_crt_dispatch@@YAHQEAUHINSTANCE__@@KQEAX@Z 0000000180004eb0 f   MSVCRT:dll_dllmain.obj
 0001:00003f00       ?dllmain_crt_process_attach@@YAHQEAUHINSTANCE__@@QEAX@Z 0000000180004f00 f   MSVCRT:dll_dllmain.obj
 0001:00004018       ?dllmain_crt_process_detach@@YAH_N@Z 0000000180005018 f   MSVCRT:dll_dllmain.obj
 0001:0000409c       ?dllmain_dispatch@@YAHQEAUHINSTANCE__@@KQEAX@Z 000000018000509c f   MSVCRT:dll_dllmain.obj
 0001:00004ab0       $$000000                   0000000180005ab0     MSVCRT:guard_dispatch.obj
 0001:00004ad0       $$000000                   0000000180005ad0     MSVCRT:guard_xfg_dispatch.obj
 0001:00004ae6       ?fin$0@?0??dllmain_crt_process_attach@@YAHQEAUHINSTANCE__@@QEAX@Z@4HA 0000000180005ae6 f   MSVCRT:dll_dllmain.obj
 0001:00004afd       ?fin$0@?0??dllmain_crt_process_detach@@YAH_N@Z@4HA 0000000180005afd f   MSVCRT:dll_dllmain.obj
 0001:00004b16       ?fin$1@?0??dllmain_crt_process_detach@@YAH_N@Z@4HA 0000000180005b16 f   MSVCRT:dll_dllmain.obj
 0001:00004b2a       ?filt$0@?0??dllmain_dispatch@@YAHQEAUHINSTANCE__@@KQEAX@Z@4HA 0000000180005b2a f   MSVCRT:dll_dllmain.obj
 0001:00004b60       __scrt_is_nonwritable_in_current_image$filt$0 0000000180005b60 f   MSVCRT:utility.obj
 0002:00000218       ?__scrt_initialize_tss_var@@3P6AHXZEA 0000000180006218     MSVCRT:thread_safe_statics.obj
 0002:00000340       ?opcLengths@@3QBEB         0000000180006340     libiterreachobj001.obj
 0002:00003638       GS_ExceptionPointers       0000000180009638     MSVCRT:gs_report.obj
 0002:00003d30       $unwind$fprintf            0000000180009d30     libiterreachobj001.obj
 0002:00003d3c       $unwind$printf             0000000180009d3c     libiterreachobj001.obj
 0002:00003d48       $unwind$?NewObject@JNIEnv_@@QEAAPEAV_jobject@@PEAV_jclass@@PEAU_jmethodID@@ZZ 0000000180009d48     libiterreachobj001.obj
 0002:00003d48       $unwind$nsk_lcomplain      0000000180009d48     libiterreachobj001.obj
 0002:00003d48       $unwind$nsk_ldisplay       0000000180009d48     libiterreachobj001.obj
 0002:00003d50       $unwind$nsk_jvmti_waitForSync 0000000180009d50     libiterreachobj001.obj
 0002:00003d50       $unwind$nsk_lvdisplay      0000000180009d50     libiterreachobj001.obj
 0002:00003d50       $unwind$_RTC_Initialize    0000000180009d50     MSVCRT:initsect.obj
 0002:00003d50       $unwind$_RTC_Terminate     0000000180009d50     MSVCRT:initsect.obj
 0002:00003d50       $unwind$?__scrt_initialize_thread_safe_statics@@YAHXZ 0000000180009d50     MSVCRT:thread_safe_statics.obj
 0002:00003d5c       $unwind$nsk_complain       0000000180009d5c     libiterreachobj001.obj
 0002:00003d5c       $unwind$nsk_printf         0000000180009d5c     libiterreachobj001.obj
 0002:00003d64       $unwind$nsk_lvcomplain     0000000180009d64     libiterreachobj001.obj
 0002:00003d7c       $unwind$nsk_ltrace         0000000180009d7c     libiterreachobj001.obj
 0002:00003d7c       $unwind$__report_gsfailure 0000000180009d7c     MSVCRT:gs_report.obj
 0002:00003d84       $unwind$nsk_lvtrace        0000000180009d84     libiterreachobj001.obj
 0002:00003d84       $unwind$__raise_securityfailure 0000000180009d84     MSVCRT:gs_report.obj
 0002:00003d84       $unwind$__scrt_initialize_crt 0000000180009d84     MSVCRT:utility.obj
 0002:00003d84       $unwind$__scrt_initialize_onexit_tables 0000000180009d84     MSVCRT:utility.obj
 0002:00003d84       $unwind$__scrt_release_startup_lock 0000000180009d84     MSVCRT:utility.obj
 0002:00003d84       $unwind$__scrt_uninitialize_crt 0000000180009d84     MSVCRT:utility.obj
 0002:00003d84       $unwind$_onexit            0000000180009d84     MSVCRT:utility.obj
 0002:00003d8c       $unwind$nsk_lverify        0000000180009d8c     libiterreachobj001.obj
 0002:00003d9c       $unwind$nsk_vprintf        0000000180009d9c     libiterreachobj001.obj
 0002:00003dac       $unwind$?nsk_jni_lverify@@YAHHPEAUJNIEnv_@@HQEBDH1ZZ 0000000180009dac     libiterreachobj001.obj
 0002:00003dc0       $unwind$?nsk_jni_check_exception@@YAHPEAUJNIEnv_@@QEBDH@Z 0000000180009dc0     libiterreachobj001.obj
 0002:00003ddc       $unwind$nsk_jvmti_parseOptions 0000000180009ddc     libiterreachobj001.obj
 0002:00003df8       $unwind$nsk_jvmti_createJVMTIEnv 0000000180009df8     libiterreachobj001.obj
 0002:00003e0c       $unwind$Java_nsk_jvmti_unit_FollowReferences_FollowRefObjects_resetTags 0000000180009e0c     libiterreachobj001.obj
 0002:00003e0c       $unwind$addRefToVerify     0000000180009e0c     libiterreachobj001.obj
 0002:00003e0c       $unwind$nsk_jvmti_resetAgentData 0000000180009e0c     libiterreachobj001.obj
 0002:00003e0c       $unwind$nsk_jvmti_resumeSync 0000000180009e0c     libiterreachobj001.obj
 0002:00003e0c       $unwind$nsk_jvmti_setFailStatus 0000000180009e0c     libiterreachobj001.obj
 0002:00003e0c       $unwind$__scrt_initialize_default_local_stdio_options 0000000180009e0c     MSVCRT:default_local_stdio_options.obj
 0002:00003e0c       $unwind$?dllmain_crt_dispatch@@YAHQEAUHINSTANCE__@@KQEAX@Z 0000000180009e0c     MSVCRT:dll_dllmain.obj
 0002:00003e0c       $unwind$DllMain            0000000180009e0c     MSVCRT:dll_dllmain_stub.obj
 0002:00003e0c       $unwind$__GSHandlerCheck   0000000180009e0c     MSVCRT:gshandler.obj
 0002:00003e0c       $unwind$?__scrt_uninitialize_thread_safe_statics@@YAXXZ 0000000180009e0c     MSVCRT:thread_safe_statics.obj
 0002:00003e0c       $unwind$__scrt_acquire_startup_lock 0000000180009e0c     MSVCRT:utility.obj
 0002:00003e0c       $unwind$__scrt_dllmain_after_initialize_c 0000000180009e0c     MSVCRT:utility.obj
 0002:00003e0c       $unwind$__scrt_dllmain_before_initialize_c 0000000180009e0c     MSVCRT:utility.obj
 0002:00003e0c       $unwind$__scrt_dllmain_crt_thread_attach 0000000180009e0c     MSVCRT:utility.obj
 0002:00003e0c       $unwind$__scrt_dllmain_crt_thread_detach 0000000180009e0c     MSVCRT:utility.obj
 0002:00003e0c       $unwind$__scrt_dllmain_uninitialize_c 0000000180009e0c     MSVCRT:utility.obj
 0002:00003e0c       $unwind$__scrt_dllmain_uninitialize_critical 0000000180009e0c     MSVCRT:utility.obj
 0002:00003e0c       $unwind$atexit             0000000180009e0c     MSVCRT:utility.obj
 0002:00003e14       $unwind$check_option       0000000180009e14     libiterreachobj001.obj
 0002:00003e14       $unwind$nsk_jvmti_findOptionValue 0000000180009e14     libiterreachobj001.obj
 0002:00003e14       $unwind$_DllMainCRTStartup 0000000180009e14     MSVCRT:dll_dllmain.obj
 0002:00003e24       $unwind$nsk_jvmti_findOptionIntValue 0000000180009e24     libiterreachobj001.obj
 0002:00003e34       $unwind$nsk_jvmti_lverify  0000000180009e34     libiterreachobj001.obj
 0002:00003e48       $unwind$exitOnError        0000000180009e48     libiterreachobj001.obj
 0002:00003e58       $unwind$Java_nsk_share_jvmti_ArgumentHandler_getAgentOptionsString 0000000180009e58     libiterreachobj001.obj
 0002:00003e6c       $unwind$Java_nsk_jvmti_unit_FollowReferences_FollowRefObjects_getTag 0000000180009e6c     libiterreachobj001.obj
 0002:00003e6c       $unwind$Java_nsk_share_jvmti_DebugeeClass_checkStatus 0000000180009e6c     libiterreachobj001.obj
 0002:00003e6c       $unwind$agentThreadWrapper 0000000180009e6c     libiterreachobj001.obj
 0002:00003e7c       $unwind$startAgentThreadWrapper 0000000180009e7c     libiterreachobj001.obj
 0002:00003e98       $unwind$syncDebuggeeStatus 0000000180009e98     libiterreachobj001.obj
 0002:00003e98       $unwind$__scrt_dllmain_exception_filter 0000000180009e98     MSVCRT:utility.obj
 0002:00003eac       $unwind$Java_nsk_share_jvmti_DebugeeClass_resetAgentData 0000000180009eac     libiterreachobj001.obj
 0002:00003eb4       $unwind$MA_checkStatus     0000000180009eb4     libiterreachobj001.obj
 0002:00003ec8       $unwind$Java_nsk_jvmti_unit_FollowReferences_FollowRefObjects_setTag 0000000180009ec8     libiterreachobj001.obj
 0002:00003ee0       $unwind$Java_nsk_jvmti_unit_FollowReferences_FollowRefObjects_addRefToVerify 0000000180009ee0     libiterreachobj001.obj
 0002:00003efc       $unwind$Agent_Initialize   0000000180009efc     libiterreachobj001.obj
 0002:00003f18       $unwind$getChainObjects    0000000180009f18     libiterreachobj001.obj
 0002:00003f34       $unwind$getTestedObjects   0000000180009f34     libiterreachobj001.obj
 0002:00003f4c       $unwind$checkTestedObjects 0000000180009f4c     libiterreachobj001.obj
 0002:00003f68       $unwind$releaseTestedObjects 0000000180009f68     libiterreachobj001.obj
 0002:00003f7c       $unwind$heapRootCallback   0000000180009f7c     libiterreachobj001.obj
 0002:00003f94       $unwind$stackReferenceCallback 0000000180009f94     libiterreachobj001.obj
 0002:00003fb0       $unwind$objectReferenceCallback 0000000180009fb0     libiterreachobj001.obj
 0002:00003fcc       $unwind$agentProc          0000000180009fcc     libiterreachobj001.obj
 0002:00003fe8       $unwind$capture_previous_context 0000000180009fe8     MSVCRT:gs_report.obj
 0002:00003ff4       $unwind$__GSHandlerCheckCommon 0000000180009ff4     MSVCRT:gshandler.obj
 0002:00004000       $xdatasym                  000000018000a000     MSVCRT:amdsecgs.obj
 0002:00004004       $unwind$?dllmain_crt_process_attach@@YAHQEAUHINSTANCE__@@QEAX@Z 000000018000a004     MSVCRT:dll_dllmain.obj
 0002:00004040       $unwind$?fin$0@?0??dllmain_crt_process_attach@@YAHQEAUHINSTANCE__@@QEAX@Z@4HA 000000018000a040     MSVCRT:dll_dllmain.obj
 0002:00004040       $unwind$?fin$0@?0??dllmain_crt_process_detach@@YAH_N@Z@4HA 000000018000a040     MSVCRT:dll_dllmain.obj
 0002:00004040       $unwind$?fin$1@?0??dllmain_crt_process_detach@@YAH_N@Z@4HA 000000018000a040     MSVCRT:dll_dllmain.obj
 0002:00004048       $unwind$?dllmain_crt_process_detach@@YAH_N@Z 000000018000a048     MSVCRT:dll_dllmain.obj
 0002:0000409c       $unwind$?dllmain_dispatch@@YAHQEAUHINSTANCE__@@KQEAX@Z 000000018000a09c     MSVCRT:dll_dllmain.obj
 0002:000040c4       $unwind$?filt$0@?0??dllmain_dispatch@@YAHQEAUHINSTANCE__@@KQEAX@Z@4HA 000000018000a0c4     MSVCRT:dll_dllmain.obj
 0002:000040cc       $unwind$__scrt_is_nonwritable_in_current_image 000000018000a0cc     MSVCRT:utility.obj
 0002:000040ec       $unwind$__scrt_is_nonwritable_in_current_image$filt$0 000000018000a0ec     MSVCRT:utility.obj
 0002:000040f4       $unwind$__scrt_fastfail    000000018000a0f4     MSVCRT:utility_desktop.obj
 0002:00004104       $unwind$__security_init_cookie 000000018000a104     MSVCRT:gs_support.obj
 0002:00004110       $unwind$__isa_available_init 000000018000a110     MSVCRT:cpu_disp.obj
 0002:00004120       $xdatasym                  000000018000a120     MSVCRT:guard_dispatch.obj
 0002:00004128       $xdatasym                  000000018000a128     MSVCRT:guard_xfg_dispatch.obj
 0002:00004130       .edata                     000000018000a130     iterreachobj001.exp
 0002:00004158       rgpv                       000000018000a158     iterreachobj001.exp
 0002:00004190       rgszName                   000000018000a190     iterreachobj001.exp
 0002:000041c8       rgwOrd                     000000018000a1c8     iterreachobj001.exp
 0002:000041e4       szName                     000000018000a1e4     iterreachobj001.exp
 0002:000041f8       $N00001                    000000018000a1f8     iterreachobj001.exp
 0002:00004207       $N00002                    000000018000a207     iterreachobj001.exp
 0002:00004214       $N00003                    000000018000a214     iterreachobj001.exp
 0002:00004259       $N00004                    000000018000a259     iterreachobj001.exp
 0002:00004296       $N00005                    000000018000a296     iterreachobj001.exp
 0002:000042de       $N00006                    000000018000a2de     iterreachobj001.exp
 0002:0000431e       $N00007                    000000018000a31e     iterreachobj001.exp
 0002:0000435b       $N00008                    000000018000a35b     iterreachobj001.exp
 0002:00004396       $N00009                    000000018000a396     iterreachobj001.exp
 0002:000043c4       $N00010                    000000018000a3c4     iterreachobj001.exp
 0002:000043f5       $N00011                    000000018000a3f5     iterreachobj001.exp
 0002:00004424       $N00012                    000000018000a424     iterreachobj001.exp
 0002:00004453       $N00013                    000000018000a453     iterreachobj001.exp
 0002:00004488       $N00014                    000000018000a488     iterreachobj001.exp
 0002:000048ea       .idata$6                   000000018000a8ea     kernel32:KERNEL32.dll
 0002:0000494e       .idata$6                   000000018000a94e     vcruntime:VCRUNTIME140.dll
 0002:00004ae0       .idata$6                   000000018000aae0     ucrt:api-ms-win-crt-heap-l1-1-0.dll
 0002:00004b00       .idata$6                   000000018000ab00     ucrt:api-ms-win-crt-runtime-l1-1-0.dll
 0002:00004b22       .idata$6                   000000018000ab22     ucrt:api-ms-win-crt-convert-l1-1-0.dll
 0002:00004b44       .idata$6                   000000018000ab44     ucrt:api-ms-win-crt-stdio-l1-1-0.dll
 0002:00004b64       .idata$6                   000000018000ab64     ucrt:api-ms-win-crt-string-l1-1-0.dll
 0003:00000000       ?codeAttributeName@@3PEBDEB 000000018000b000     libiterreachobj001.obj
 0003:00000008       ?lineNumberAttributeName@@3PEBDEB 000000018000b008     libiterreachobj001.obj
 0003:00000010       ?localVarAttributeName@@3PEBDEB 000000018000b010     libiterreachobj001.obj
 0003:00000018       ?localVarTypeAttributeName@@3PEBDEB 000000018000b018     libiterreachobj001.obj
 0003:00000020       ?stackMapAttributeName@@3PEBDEB 000000018000b020     libiterreachobj001.obj
 0003:00000028       ?callBytes@@3PAEA          000000018000b028     libiterreachobj001.obj
 0003:0000002c       ?allocBytes@@3PAEA         000000018000b02c     libiterreachobj001.obj
 0003:0001aad4       redefineAttempted          0000000180025ad4     libiterreachobj001.obj
 0003:0001aad8       nsk_context                0000000180025ad8     libiterreachobj001.obj
 0003:0001aae4       redefineSucceed            0000000180025ae4     libiterreachobj001.obj
 0003:0001aae8       agentFailed                0000000180025ae8     libiterreachobj001.obj
 0003:0001aaec       currentAgentStatus         0000000180025aec     libiterreachobj001.obj
 0003:0001aaf0       context                    0000000180025af0     libiterreachobj001.obj
 0003:0001aba8       agentThread                0000000180025ba8     libiterreachobj001.obj
 0003:0001abb0       agentThreadProc            0000000180025bb0     libiterreachobj001.obj
 0003:0001abb8       agentThreadArg             0000000180025bb8     libiterreachobj001.obj
 0003:0001abc0       agent_data                 0000000180025bc0     libiterreachobj001.obj
 0003:0001abd0       jvmti_env                  0000000180025bd0     libiterreachobj001.obj
 0003:0001abd8       jvm                        0000000180025bd8     libiterreachobj001.obj
 0003:0001abe0       jni_env                    0000000180025be0     libiterreachobj001.obj
 0003:0001abe8       checkStatus_func           0000000180025be8     libiterreachobj001.obj
 0003:0001abf0       ?codeAttributeIndex@@3GA   0000000180025bf0     libiterreachobj001.obj
 0003:0001abf4       ?lineNumberAttributeIndex@@3GA 0000000180025bf4     libiterreachobj001.obj
 0003:0001abf8       ?localVarAttributeIndex@@3GA 0000000180025bf8     libiterreachobj001.obj
 0003:0001abfc       ?localVarTypeAttributeIndex@@3GA 0000000180025bfc     libiterreachobj001.obj
 0003:0001ac00       ?stackMapAttributeIndex@@3GA 0000000180025c00     libiterreachobj001.obj
 0003:0001ac04       ?stackFrameOffset@@3GA     0000000180025c04     libiterreachobj001.obj
 0003:0001ac08       ?mode@@3HA                 0000000180025c08     libiterreachobj001.obj
 0003:0001ac0c       ?constantPoolSize@@3GA     0000000180025c0c     libiterreachobj001.obj
 0003:0001ac10       ?orig@@3PEBEEB             0000000180025c10     libiterreachobj001.obj
 0003:0001ac18       ?gen@@3PEAEEA              0000000180025c18     libiterreachobj001.obj
 0003:0001ac20       ?inputPos@@3PEAEEA         0000000180025c20     libiterreachobj001.obj
 0003:0001ac28       ?endPos@@3PEBEEB           0000000180025c28     libiterreachobj001.obj
 0003:0001ac30       ?genPos@@3PEAEEA           0000000180025c30     libiterreachobj001.obj
 0003:0001ac38       ?markPos@@3PEAEEA          0000000180025c38     libiterreachobj001.obj
 0003:0001ac40       ?constantPool@@3PEAPEADEA  0000000180025c40     libiterreachobj001.obj
 0003:0001ac48       ?constantPoolCount@@3GA    0000000180025c48     libiterreachobj001.obj
 0003:0001ac4c       ?zeroBytes@@3PAEA          0000000180025c4c     libiterreachobj001.obj
 0003:0001ac50       ?codeLength@@3IA           0000000180025c50     libiterreachobj001.obj
 0003:0001ac54       info                       0000000180025c54     libiterreachobj001.obj
 0003:0001ac58       ?map@@3PEAIEA              0000000180025c58     libiterreachobj001.obj
 0003:0001ac60       ?widening@@3PEACEA         0000000180025c60     libiterreachobj001.obj
 0003:0001ac68       timeout                    0000000180025c68     libiterreachobj001.obj
 0003:0001ac70       chainLength                0000000180025c70     libiterreachobj001.obj
 0003:0001ac74       objectsCount               0000000180025c74     libiterreachobj001.obj
 0003:0001ac78       objectDescList             0000000180025c78     libiterreachobj001.obj
 0003:0001ac80       fakeUserData               0000000180025c80     libiterreachobj001.obj
 0003:0001ac84       userDataError              0000000180025c84     libiterreachobj001.obj
 0003:0001ac90       GS_ExceptionRecord         0000000180025c90     MSVCRT:gs_report.obj
 0003:0001ad30       GS_ContextRecord           0000000180025d30     MSVCRT:gs_report.obj
 0003:0001b200       ?g_tss_cv@@3U_RTL_CONDITION_VARIABLE@@A 0000000180026200     MSVCRT:thread_safe_statics.obj
 0003:0001b208       ?g_tss_event@@3PEAXEA      0000000180026208     MSVCRT:thread_safe_statics.obj
 0003:0001b210       ?g_tss_mutex@@3U_RTL_CRITICAL_SECTION@@A 0000000180026210     MSVCRT:thread_safe_statics.obj
 0003:0001b238       ?g_sleep_condition_variable_cs@@3P6AHPEAU_RTL_CONDITION_VARIABLE@@PEAU_RTL_CRITICAL_SECTION@@K@ZEA 0000000180026238     MSVCRT:thread_safe_statics.obj
 0003:0001b240       ?g_wake_all_condition_variable@@3P6AXPEAU_RTL_CONDITION_VARIABLE@@@ZEA 0000000180026240     MSVCRT:thread_safe_statics.obj
 0003:0001b24c       ?__proc_attached@@3HA      000000018002624c     MSVCRT:dll_dllmain.obj
 0003:0001b260       ?is_initialized_as_dll@@3_NA 0000000180026260     MSVCRT:utility.obj
 0003:0001b261       ?module_local_atexit_table_initialized@@3_NA 0000000180026261     MSVCRT:utility.obj
 0003:0001b268       ?module_local_atexit_table@@3U_onexit_table_t@@A 0000000180026268     MSVCRT:utility.obj
 0003:0001b280       ?module_local_at_quick_exit_table@@3U_onexit_table_t@@A 0000000180026280     MSVCRT:utility.obj
